ELF Header:
  Magic:   7f 45 4c 46 01 01 01 00 00 00 00 00 00 00 00 00 
  Class:                             ELF32
  Data:                              2's complement, little endian
  Version:                           1 (current)
  OS/ABI:                            UNIX - System V
  ABI Version:                       0
  Type:                              EXEC (Executable file)
  Machine:                           CSKY
  Version:                           0x1
  Entry point address:               0x10c
  Start of program headers:          52 (bytes into file)
  Start of section headers:          304444 (bytes into file)
  Flags:                             0x21000000
  Size of this header:               52 (bytes)
  Size of program headers:           32 (bytes)
  Number of program headers:         2
  Size of section headers:           40 (bytes)
  Number of section headers:         152
  Section header string table index: 149

Section Headers:
  [Nr] Name              Type            Addr     Off    Size   ES Flg Lk Inf Al
  [ 0]                   NULL            00000000 000000 000000 00      0   0  0
  [ 1] .text             PROGBITS        00000000 001000 001a50 00  AX  0   0 1024
  [ 2] .text.__main      PROGBITS        00001a50 002a50 000038 00  AX  0   0  4
  [ 3] .text.SYSCON_Gene PROGBITS        00001a88 002a88 000074 00  AX  0   0  4
  [ 4] .text.SYSCON_RST_ PROGBITS        00001afc 002afc 00004c 00  AX  0   0  4
  [ 5] .text.SYSCON_Gene PROGBITS        00001b48 002b48 000030 00  AX  0   0  4
  [ 6] .text.SystemCLK_H PROGBITS        00001b78 002b78 000088 00  AX  0   0  4
  [ 7] .text.SYSCON_HFOS PROGBITS        00001c00 002c00 000028 00  AX  0   0  4
  [ 8] .text.SYSCON_WDT_ PROGBITS        00001c28 002c28 00003c 00  AX  0   0  4
  [ 9] .text.SYSCON_IWDC PROGBITS        00001c64 002c64 000014 00  AX  0   0  4
  [10] .text.SYSCON_IWDC PROGBITS        00001c78 002c78 000018 00  AX  0   0  4
  [11] .text.SYSCON_LVD_ PROGBITS        00001c90 002c90 000020 00  AX  0   0  4
  [12] .text.LVD_Int_Ena PROGBITS        00001cb0 002cb0 00001c 00  AX  0   0  4
  [13] .text.IWDT_Int_En PROGBITS        00001ccc 002ccc 00001c 00  AX  0   0  4
  [14] .text.EXTI_trigge PROGBITS        00001ce8 002ce8 000040 00  AX  0   0  4
  [15] .text.EXTI_interr PROGBITS        00001d28 002d28 000034 00  AX  0   0  4
  [16] .text.GPIO_EXTI_i PROGBITS        00001d5c 002d5c 000004 00  AX  0   0  2
  [17] .text.EXI4_Int_En PROGBITS        00001d60 002d60 000010 00  AX  0   0  4
  [18] .text.SYSCON_Int_ PROGBITS        00001d70 002d70 00000c 00  AX  0   0  4
  [19] .text.SYSCON_Int_ PROGBITS        00001d7c 002d7c 00000c 00  AX  0   0  4
  [20] .text.SYSCON_INT_ PROGBITS        00001d88 002d88 000024 00  AX  0   0  4
  [21] .text.Set_INT_Pri PROGBITS        00001dac 002dac 000030 00  AX  0   0  4
  [22] .text.GPIO_Init   PROGBITS        00001ddc 002ddc 0000e0 00  AX  0   0  4
  [23] .text.GPIO_PullHi PROGBITS        00001ebc 002ebc 000014 00  AX  0   0  2
  [24] .text.GPIO_DriveS PROGBITS        00001ed0 002ed0 00000e 00  AX  0   0  2
  [25] .text.GPIO_IntGro PROGBITS        00001ee0 002ee0 00010c 00  AX  0   0  4
  [26] .text.GPIOA0_EXI_ PROGBITS        00001fec 002fec 0000fc 00  AX  0   0  4
  [27] .text.GPIO_Write_ PROGBITS        000020e8 0030e8 000008 00  AX  0   0  2
  [28] .text.GPIO_Write_ PROGBITS        000020f0 0030f0 000008 00  AX  0   0  2
  [29] .text.GPIO_Revers PROGBITS        000020f8 0030f8 000016 00  AX  0   0  2
  [30] .text.GPIO_Read_S PROGBITS        0000210e 00310e 000010 00  AX  0   0  2
  [31] .text.LPT_Soft_Re PROGBITS        00002120 003120 000014 00  AX  0   0  4
  [32] .text.WWDT_CNT_Lo PROGBITS        00002134 003134 000010 00  AX  0   0  4
  [33] .text.BT_DeInit   PROGBITS        00002144 003144 00001c 00  AX  0   0  2
  [34] .text.BT_Start    PROGBITS        00002160 003160 000008 00  AX  0   0  2
  [35] .text.BT_Soft_Res PROGBITS        00002168 003168 00000a 00  AX  0   0  2
  [36] .text.BT_Configur PROGBITS        00002172 003172 000018 00  AX  0   0  2
  [37] .text.BT_ControlS PROGBITS        0000218a 00318a 00002c 00  AX  0   0  2
  [38] .text.BT_Period_C PROGBITS        000021b6 0031b6 000006 00  AX  0   0  2
  [39] .text.BT_ConfigIn PROGBITS        000021bc 0031bc 000012 00  AX  0   0  2
  [40] .text.BT1_INT_ENA PROGBITS        000021d0 0031d0 000010 00  AX  0   0  4
  [41] .text.GPT_IO_Init PROGBITS        000021e0 0031e0 0000a0 00  AX  0   0  4
  [42] .text.GPT_Configu PROGBITS        00002280 003280 000014 00  AX  0   0  4
  [43] .text.GPT_WaveCtr PROGBITS        00002294 003294 000044 00  AX  0   0  4
  [44] .text.GPT_WaveLoa PROGBITS        000022d8 0032d8 000014 00  AX  0   0  4
  [45] .text.GPT_WaveOut PROGBITS        000022ec 0032ec 0000b4 00  AX  0   0  4
  [46] .text.GPT_Start   PROGBITS        000023a0 0033a0 000010 00  AX  0   0  4
  [47] .text.GPT_Period_ PROGBITS        000023b0 0033b0 000010 00  AX  0   0  4
  [48] .text.GPT_ConfigI PROGBITS        000023c0 0033c0 00001c 00  AX  0   0  4
  [49] .text.UART0_DeIni PROGBITS        000023dc 0033dc 000018 00  AX  0   0  4
  [50] .text.UART1_DeIni PROGBITS        000023f4 0033f4 000018 00  AX  0   0  4
  [51] .text.UART2_DeIni PROGBITS        0000240c 00340c 000018 00  AX  0   0  4
  [52] .text.UART1_Int_E PROGBITS        00002424 003424 00001c 00  AX  0   0  4
  [53] .text.UART2_Int_E PROGBITS        00002440 003440 00001c 00  AX  0   0  4
  [54] .text.UART_IO_Ini PROGBITS        0000245c 00345c 0000ec 00  AX  0   0  4
  [55] .text.UARTInitRxT PROGBITS        00002548 003548 000010 00  AX  0   0  4
  [56] .text.UARTTransmi PROGBITS        00002558 003558 00001e 00  AX  0   0  2
  [57] .text.EPT_Stop    PROGBITS        00002578 003578 000028 00  AX  0   0  4
  [58] .text.startup.mai PROGBITS        000025a0 0035a0 000024 00  AX  0   0  4
  [59] .text.delay_nms   PROGBITS        000025c4 0035c4 00002c 00  AX  0   0  2
  [60] .text.delay_nus   PROGBITS        000025f0 0035f0 000022 00  AX  0   0  2
  [61] .text.BT_CONFIG   PROGBITS        00002614 003614 000060 00  AX  0   0  4
  [62] .text.SYSCON_CONF PROGBITS        00002674 003674 000062 00  AX  0   0  2
  [63] .text.APT32F102_i PROGBITS        000026d8 0036d8 00004c 00  AX  0   0  4
  [64] .text.SYSCONIntHa PROGBITS        00002724 003724 0000f0 00  AX  0   0  4
  [65] .text.IFCIntHandl PROGBITS        00002814 003814 000068 00  AX  0   0  4
  [66] .text.ADCIntHandl PROGBITS        0000287c 00387c 000068 00  AX  0   0  4
  [67] .text.EPT0IntHand PROGBITS        000028e4 0038e4 0001ac 00  AX  0   0  4
  [68] .text.WWDTHandler PROGBITS        00002a90 003a90 000034 00  AX  0   0  4
  [69] .text.GPT0IntHand PROGBITS        00002ac4 003ac4 000080 00  AX  0   0  4
  [70] .text.RTCIntHandl PROGBITS        00002b44 003b44 000070 00  AX  0   0  4
  [71] .text.UART0IntHan PROGBITS        00002bb4 003bb4 00003c 00  AX  0   0  4
  [72] .text.UART1IntHan PROGBITS        00002bf0 003bf0 000094 00  AX  0   0  4
  [73] .text.UART2IntHan PROGBITS        00002c84 003c84 00004c 00  AX  0   0  4
  [74] .text.SPI0IntHand PROGBITS        00002cd0 003cd0 0000e8 00  AX  0   0  4
  [75] .text.SIO0IntHand PROGBITS        00002db8 003db8 000054 00  AX  0   0  4
  [76] .text.EXI0IntHand PROGBITS        00002e0c 003e0c 000030 00  AX  0   0  4
  [77] .text.EXI1IntHand PROGBITS        00002e3c 003e3c 000030 00  AX  0   0  4
  [78] .text.EXI2to3IntH PROGBITS        00002e6c 003e6c 000048 00  AX  0   0  4
  [79] .text.EXI4to9IntH PROGBITS        00002eb4 003eb4 000020 00  AX  0   0  4
  [80] .text.EXI10to15In PROGBITS        00002ed4 003ed4 00006c 00  AX  0   0  4
  [81] .text.LPTIntHandl PROGBITS        00002f40 003f40 000034 00  AX  0   0  4
  [82] .text.BT0IntHandl PROGBITS        00002f74 003f74 00004c 00  AX  0   0  4
  [83] .text.BT1IntHandl PROGBITS        00002fc0 003fc0 000070 00  AX  0   0  4
  [84] .text.PriviledgeV PROGBITS        00003030 004030 000002 00  AX  0   0  2
  [85] .text.PendTrapHan PROGBITS        00003032 004032 000008 00  AX  0   0  2
  [86] .text.Trap3Handle PROGBITS        0000303a 00403a 000008 00  AX  0   0  2
  [87] .text.Trap2Handle PROGBITS        00003042 004042 000008 00  AX  0   0  2
  [88] .text.Trap1Handle PROGBITS        0000304a 00404a 000008 00  AX  0   0  2
  [89] .text.Trap0Handle PROGBITS        00003052 004052 000008 00  AX  0   0  2
  [90] .text.UnrecExecpH PROGBITS        0000305a 00405a 000008 00  AX  0   0  2
  [91] .text.BreakPointH PROGBITS        00003062 004062 000008 00  AX  0   0  2
  [92] .text.AccessErrHa PROGBITS        0000306a 00406a 000008 00  AX  0   0  2
  [93] .text.IllegalInst PROGBITS        00003072 004072 000008 00  AX  0   0  2
  [94] .text.MisalignedH PROGBITS        0000307a 00407a 000008 00  AX  0   0  2
  [95] .text.CNTAIntHand PROGBITS        00003082 004082 000008 00  AX  0   0  2
  [96] .text.I2CIntHandl PROGBITS        0000308a 00408a 000008 00  AX  0   0  2
  [97] .text.__divsi3    PROGBITS        00003094 004094 000024 00  AX  0   0  4
  [98] .text.__udivsi3   PROGBITS        000030b8 0040b8 000024 00  AX  0   0  4
  [99] .text.__umodsi3   PROGBITS        000030dc 0040dc 000024 00  AX  0   0  4
  [100] .text.CK_CPU_EnAl PROGBITS        00003100 004100 000006 00  AX  0   0  2
  [101] .text.CK_CPU_DisA PROGBITS        00003106 004106 000006 00  AX  0   0  2
  [102] .text.UARTx_Init  PROGBITS        0000310c 00410c 000120 00  AX  0   0  4
  [103] .text.UART1_RecvI PROGBITS        0000322c 00422c 000034 00  AX  0   0  4
  [104] .text.UART1_TASK  PROGBITS        00003260 004260 000060 00  AX  0   0  4
  [105] .text.BUS485_Send PROGBITS        000032c0 0042c0 0000c4 00  AX  0   0  4
  [106] .text.MultSend_Ta PROGBITS        00003384 004384 000064 00  AX  0   0  4
  [107] .text.Set_GroupSe PROGBITS        000033e8 0043e8 00005c 00  AX  0   0  4
  [108] .text.BUS485Send_ PROGBITS        00003444 004444 00002c 00  AX  0   0  4
  [109] .text.BusIdle_Tas PROGBITS        00003470 004470 00003c 00  AX  0   0  4
  [110] .text.BusBusy_Tas PROGBITS        000034ac 0044ac 000054 00  AX  0   0  4
  [111] .text.Dbg_Println PROGBITS        00003500 004500 00000c 00  AX  0   0  2
  [112] .text.DIP_GetSwit PROGBITS        0000350c 00450c 000034 00  AX  0   0  4
  [113] .text.DIP_Switch_ PROGBITS        00003540 004540 00008c 00  AX  0   0  4
  [114] .text.DIP_ScanTas PROGBITS        000035cc 0045cc 00008c 00  AX  0   0  4
  [115] .text.Relay_Init  PROGBITS        00003658 004658 0000cc 00  AX  0   0  4
  [116] .text.CheckSum    PROGBITS        00003724 004724 000016 00  AX  0   0  2
  [117] .text.Change_OUTV PROGBITS        0000373c 00473c 00001c 00  AX  0   0  4
  [118] .text.BLV_VolOut_ PROGBITS        00003758 004758 000090 00  AX  0   0  4
  [119] .text.BLV_RLY_Ctr PROGBITS        000037e8 0047e8 00007c 00  AX  0   0  4
  [120] .text.BLV_RLY_Tas PROGBITS        00003864 004864 000054 00  AX  0   0  4
  [121] .text.BLV_A9RLY_C PROGBITS        000038b8 0048b8 00009c 00  AX  0   0  4
  [122] .text.BLV_A9RLY_C PROGBITS        00003954 004954 000078 00  AX  0   0  4
  [123] .text.BLV_RLY_RS4 PROGBITS        000039cc 0049cc 0000b0 00  AX  0   0  4
  [124] .text.TK_Sampling PROGBITS        00003a7c 004a7c 000058 00  AX  0   0  4
  [125] .text.TKEYIntHand PROGBITS        00003ad4 004ad4 000088 00  AX  0   0  4
  [126] .text.get_key_num PROGBITS        00003b5c 004b5c 000028 00  AX  0   0  4
  [127] .text.TK_Scan_Sta PROGBITS        00003b84 004b84 000020 00  AX  0   0  4
  [128] .text.TK_Keymap_p PROGBITS        00003ba4 004ba4 000180 00  AX  0   0  4
  [129] .text.TK_overflow PROGBITS        00003d24 004d24 00011c 00  AX  0   0  4
  [130] .text.TK_Baseline PROGBITS        00003e40 004e40 0001d0 00  AX  0   0  4
  [131] .text.TK_result_p PROGBITS        00004010 005010 000054 00  AX  0   0  4
  [132] .text.CORETHandle PROGBITS        00004064 005064 000078 00  AX  0   0  4
  [133] .text.std_clk_cal PROGBITS        000040dc 0050dc 000284 00  AX  0   0  4
  [134] .RomCode          PROGBITS        00004360 00609c 000000 00   W  0   0  1
  [135] .rodata           PROGBITS        00004360 005360 000200 00   A  0   0  4
  [136] .data             PROGBITS        20000000 006000 00009c 00  WA  0   0  4
  [137] .bss              NOBITS          2000009c 00609c 0005ac 00  WA  0   0  4
  [138] .csky.attributes  CSKY_ATTRIBUTES 00000000 00609c 000022 00      0   0  1
  [139] .comment          PROGBITS        00000000 0060be 000042 01  MS  0   0  1
  [140] .csky_stack_size  PROGBITS        00000000 006100 0007bc 00      0   0 16
  [141] .debug_line       PROGBITS        00000000 0068bc 0035d5 00      0   0  1
  [142] .debug_info       PROGBITS        00000000 009e91 02a208 00      0   0  1
  [143] .debug_abbrev     PROGBITS        00000000 034099 0026cf 00      0   0  1
  [144] .debug_aranges    PROGBITS        00000000 036768 000c10 00      0   0  8
  [145] .debug_ranges     PROGBITS        00000000 037378 000b58 00      0   0  1
  [146] .debug_str        PROGBITS        00000000 037ed0 008721 01  MS  0   0  1
  [147] .debug_frame      PROGBITS        00000000 0405f4 001bec 00      0   0  4
  [148] .debug_loc        PROGBITS        00000000 0421e0 002c1e 00      0   0  1
  [149] .shstrtab         STRTAB          00000000 04990b 000c30 00      0   0  1
  [150] .symtab           SYMTAB          00000000 044e00 003920 10     151 631  4
  [151] .strtab           STRTAB          00000000 048720 0011eb 00      0   0  1
Key to Flags:
  W (write), A (alloc), X (execute), M (merge), S (strings), I (info),
  L (link order), O (extra OS processing required), G (group), T (TLS),
  C (compressed), x (unknown), o (OS specific), E (exclude),
  p (processor specific)

Program Headers:
  Type           Offset   VirtAddr   PhysAddr   FileSiz MemSiz  Flg Align
  LOAD           0x001000 0x00000000 0x00000000 0x04560 0x04560 R E 0x1000
  LOAD           0x006000 0x20000000 0x00004560 0x0009c 0x00648 RW  0x1000

 Section to Segment mapping:
  Segment Sections...
   00     .text .text.__main .text.SYSCON_General_CMD.part.0 .text.SYSCON_RST_VALUE .text.SYSCON_General_CMD .text.SystemCLK_HCLKDIV_PCLKDIV_Config .text.SYSCON_HFOSC_SELECTE .text.SYSCON_WDT_CMD .text.SYSCON_IWDCNT_Reload .text.SYSCON_IWDCNT_Config .text.SYSCON_LVD_Config .text.LVD_Int_Enable .text.IWDT_Int_Enable .text.EXTI_trigger_CMD .text.EXTI_interrupt_CMD .text.GPIO_EXTI_interrupt .text.EXI4_Int_Enable .text.SYSCON_Int_Enable .text.SYSCON_Int_Disable .text.SYSCON_INT_Priority .text.Set_INT_Priority .text.GPIO_Init .text.GPIO_PullHigh_Init .text.GPIO_DriveStrength_EN .text.GPIO_IntGroup_Set .text.GPIOA0_EXI_Init .text.GPIO_Write_High .text.GPIO_Write_Low .text.GPIO_Reverse .text.GPIO_Read_Status .text.LPT_Soft_Reset .text.WWDT_CNT_Load .text.BT_DeInit .text.BT_Start .text.BT_Soft_Reset .text.BT_Configure .text.BT_ControlSet_Configure .text.BT_Period_CMP_Write .text.BT_ConfigInterrupt_CMD .text.BT1_INT_ENABLE .text.GPT_IO_Init .text.GPT_Configure .text.GPT_WaveCtrl_Configure .text.GPT_WaveLoad_Configure .text.GPT_WaveOut_Configure .text.GPT_Start .text.GPT_Period_CMP_Write .text.GPT_ConfigInterrupt_CMD .text.UART0_DeInit .text.UART1_DeInit .text.UART2_DeInit .text.UART1_Int_Enable .text.UART2_Int_Enable .text.UART_IO_Init .text.UARTInitRxTxIntEn .text.UARTTransmit .text.EPT_Stop .text.startup.main .text.delay_nms .text.delay_nus .text.BT_CONFIG .text.SYSCON_CONFIG .text.APT32F102_init .text.SYSCONIntHandler .text.IFCIntHandler .text.ADCIntHandler .text.EPT0IntHandler .text.WWDTHandler .text.GPT0IntHandler .text.RTCIntHandler .text.UART0IntHandler .text.UART1IntHandler .text.UART2IntHandler .text.SPI0IntHandler .text.SIO0IntHandler .text.EXI0IntHandler .text.EXI1IntHandler .text.EXI2to3IntHandler .text.EXI4to9IntHandler .text.EXI10to15IntHandler .text.LPTIntHandler .text.BT0IntHandler .text.BT1IntHandler .text.PriviledgeVioHandler .text.PendTrapHandler .text.Trap3Handler .text.Trap2Handler .text.Trap1Handler .text.Trap0Handler .text.UnrecExecpHandler .text.BreakPointHandler .text.AccessErrHandler .text.IllegalInstrHandler .text.MisalignedHandler .text.CNTAIntHandler .text.I2CIntHandler .text.__divsi3 .text.__udivsi3 .text.__umodsi3 .text.CK_CPU_EnAllNormalIrq .text.CK_CPU_DisAllNormalIrq .text.UARTx_Init .text.UART1_RecvINT_Processing .text.UART1_TASK .text.BUS485_Send .text.MultSend_Task .text.Set_GroupSend .text.BUS485Send_Task .text.BusIdle_Task .text.BusBusy_Task .text.Dbg_Println .text.DIP_GetSwitchState .text.DIP_Switch_Init .text.DIP_ScanTask .text.Relay_Init .text.CheckSum .text.Change_OUTV .text.BLV_VolOut_Ctrl .text.BLV_RLY_Ctrl_Purpose .text.BLV_RLY_Task .text.BLV_A9RLY_CMD_SET_Processing .text.BLV_A9RLY_CMD_READ_Processing .text.BLV_RLY_RS485_Pro .text.TK_Sampling_prog .text.TKEYIntHandler .text.get_key_number .text.TK_Scan_Start .text.TK_Keymap_prog .text.TK_overflow_predict .text.TK_Baseline_tracking .text.TK_result_prog .text.CORETHandler .text.std_clk_calib .rodata 
   01     .data .bss 
======================================================================
Csky GNU Linker

======================================================================

Section Cross References

	Obj/mcu_initial.o(.text.SYSCON_CONFIG) refers to Obj/FWlib_apt32f102_syscon.o(.text.SYSCON_RST_VALUE) for SYSCON_RST_VALUE
	Obj/FWlib_apt32f102_syscon.o(.text.SYSCON_HFOSC_SELECTE) refers to Obj/FWlib_apt32f102_syscon.o(.text.SYSCON_General_CMD) for SYSCON_General_CMD
	Obj/mcu_initial.o(.text.SYSCON_CONFIG) refers to Obj/FWlib_apt32f102_syscon.o(.text.SYSCON_General_CMD) for SYSCON_General_CMD
	Obj/mcu_initial.o(.text.SYSCON_CONFIG) refers to Obj/FWlib_apt32f102_syscon.o(.text.SystemCLK_HCLKDIV_PCLKDIV_Config) for SystemCLK_HCLKDIV_PCLKDIV_Config
	Obj/mcu_initial.o(.text.SYSCON_CONFIG) refers to Obj/FWlib_apt32f102_syscon.o(.text.SYSCON_HFOSC_SELECTE) for SYSCON_HFOSC_SELECTE
	Obj/mcu_initial.o(.text.SYSCON_CONFIG) refers to Obj/FWlib_apt32f102_syscon.o(.text.SYSCON_WDT_CMD) for SYSCON_WDT_CMD
	Obj/main.o(.text.startup.main) refers to Obj/FWlib_apt32f102_syscon.o(.text.SYSCON_IWDCNT_Reload) for SYSCON_IWDCNT_Reload
	Obj/mcu_initial.o(.text.delay_nms) refers to Obj/FWlib_apt32f102_syscon.o(.text.SYSCON_IWDCNT_Reload) for SYSCON_IWDCNT_Reload
	Obj/mcu_initial.o(.text.SYSCON_CONFIG) refers to Obj/FWlib_apt32f102_syscon.o(.text.SYSCON_IWDCNT_Reload) for SYSCON_IWDCNT_Reload
	Obj/mcu_initial.o(.text.SYSCON_CONFIG) refers to Obj/FWlib_apt32f102_syscon.o(.text.SYSCON_IWDCNT_Config) for SYSCON_IWDCNT_Config
	Obj/mcu_initial.o(.text.SYSCON_CONFIG) refers to Obj/FWlib_apt32f102_syscon.o(.text.SYSCON_LVD_Config) for SYSCON_LVD_Config
	Obj/mcu_initial.o(.text.SYSCON_CONFIG) refers to Obj/FWlib_apt32f102_syscon.o(.text.LVD_Int_Enable) for LVD_Int_Enable
	Obj/mcu_initial.o(.text.SYSCON_CONFIG) refers to Obj/FWlib_apt32f102_syscon.o(.text.IWDT_Int_Enable) for IWDT_Int_Enable
	Obj/mcu_interrupt.o(.text.EPT0IntHandler) refers to Obj/FWlib_apt32f102_syscon.o(.text.EXTI_trigger_CMD) for EXTI_trigger_CMD
	Obj/SYSTEM_uart.o(.text.UARTx_Init) refers to Obj/FWlib_apt32f102_syscon.o(.text.EXTI_trigger_CMD) for EXTI_trigger_CMD
	Obj/SYSTEM_uart.o(.text.UARTx_Init) refers to Obj/FWlib_apt32f102_syscon.o(.text.EXTI_interrupt_CMD) for EXTI_interrupt_CMD
	Obj/SYSTEM_uart.o(.text.UARTx_Init) refers to Obj/FWlib_apt32f102_syscon.o(.text.GPIO_EXTI_interrupt) for GPIO_EXTI_interrupt
	Obj/SYSTEM_uart.o(.text.UARTx_Init) refers to Obj/FWlib_apt32f102_syscon.o(.text.EXI4_Int_Enable) for EXI4_Int_Enable
	Obj/mcu_initial.o(.text.SYSCON_CONFIG) refers to Obj/FWlib_apt32f102_syscon.o(.text.SYSCON_Int_Enable) for SYSCON_Int_Enable
	Obj/SYSTEM_uart.o(.text.UART1_TASK) refers to Obj/FWlib_apt32f102_syscon.o(.text.SYSCON_Int_Enable) for SYSCON_Int_Enable
	Obj/SYSTEM_uart.o(.text.UART1_TASK) refers to Obj/FWlib_apt32f102_syscon.o(.text.SYSCON_Int_Disable) for SYSCON_Int_Disable
	Obj/mcu_initial.o(.text.APT32F102_init) refers to Obj/FWlib_apt32f102_syscon.o(.text.SYSCON_INT_Priority) for SYSCON_INT_Priority
	Obj/mcu_initial.o(.text.APT32F102_init) refers to Obj/FWlib_apt32f102_syscon.o(.text.Set_INT_Priority) for Set_INT_Priority
	Obj/SYSTEM_uart.o(.text.UARTx_Init) refers to Obj/FWlib_apt32f102_gpio.o(.text.GPIO_Write_Low) for GPIO_Write_Low
	Obj/SYSTEM_uart.o(.text.BUS485_Send) refers to Obj/FWlib_apt32f102_gpio.o(.text.GPIO_Write_Low) for GPIO_Write_Low
	Obj/SYSTEM_control_rly.o(.text.BLV_RLY_Ctrl_Purpose) refers to Obj/FWlib_apt32f102_gpio.o(.text.GPIO_Write_Low) for GPIO_Write_Low
	Obj/SYSTEM_uart.o(.text.BUS485_Send) refers to Obj/FWlib_apt32f102_gpio.o(.text.GPIO_Reverse) for GPIO_Reverse
	Obj/SYSTEM_uart.o(.text.BusBusy_Task) refers to Obj/FWlib_apt32f102_gpio.o(.text.GPIO_Read_Status) for GPIO_Read_Status
	Obj/SYSTEM_dip_switch.o(.text.DIP_GetSwitchState) refers to Obj/FWlib_apt32f102_gpio.o(.text.GPIO_Read_Status) for GPIO_Read_Status
	Obj/SYSTEM_uart.o(.text.UARTx_Init) refers to Obj/FWlib_apt32f102_gpio.o(.text.GPIO_Init) for GPIO_Init
	Obj/SYSTEM_dip_switch.o(.text.DIP_Switch_Init) refers to Obj/FWlib_apt32f102_gpio.o(.text.GPIO_Init) for GPIO_Init
	Obj/SYSTEM_control_rly.o(.text.Relay_Init) refers to Obj/FWlib_apt32f102_gpio.o(.text.GPIO_Init) for GPIO_Init
	Obj/SYSTEM_uart.o(.text.UARTx_Init) refers to Obj/FWlib_apt32f102_gpio.o(.text.GPIO_PullHigh_Init) for GPIO_PullHigh_Init
	Obj/SYSTEM_dip_switch.o(.text.DIP_Switch_Init) refers to Obj/FWlib_apt32f102_gpio.o(.text.GPIO_PullHigh_Init) for GPIO_PullHigh_Init
	Obj/SYSTEM_uart.o(.text.UARTx_Init) refers to Obj/FWlib_apt32f102_gpio.o(.text.GPIO_DriveStrength_EN) for GPIO_DriveStrength_EN
	Obj/SYSTEM_uart.o(.text.UARTx_Init) refers to Obj/FWlib_apt32f102_gpio.o(.text.GPIO_IntGroup_Set) for GPIO_IntGroup_Set
	Obj/SYSTEM_uart.o(.text.UARTx_Init) refers to Obj/FWlib_apt32f102_gpio.o(.text.GPIOA0_EXI_Init) for GPIOA0_EXI_Init
	Obj/SYSTEM_uart.o(.text.BUS485_Send) refers to Obj/FWlib_apt32f102_gpio.o(.text.GPIO_Write_High) for GPIO_Write_High
	Obj/SYSTEM_control_rly.o(.text.Relay_Init) refers to Obj/FWlib_apt32f102_gpio.o(.text.GPIO_Write_High) for GPIO_Write_High
	Obj/SYSTEM_control_rly.o(.text.BLV_RLY_Ctrl_Purpose) refers to Obj/FWlib_apt32f102_gpio.o(.text.GPIO_Write_High) for GPIO_Write_High
	FWlib_apt32f102_clkcalib.o(.text.std_clk_calib) refers to Obj/FWlib_apt32f102_lpt.o(.text.LPT_Soft_Reset) for LPT_Soft_Reset
	Obj/mcu_interrupt.o(.text.WWDTHandler) refers to Obj/FWlib_apt32f102_wwdt.o(.text.WWDT_CNT_Load) for WWDT_CNT_Load
	Obj/mcu_initial.o(.text.BT_CONFIG) refers to Obj/FWlib_apt32f102_bt.o(.text.BT_DeInit) for BT_DeInit
	Obj/mcu_initial.o(.text.BT_CONFIG) refers to Obj/FWlib_apt32f102_bt.o(.text.BT_Start) for BT_Start
	FWlib_apt32f102_clkcalib.o(.text.std_clk_calib) refers to Obj/FWlib_apt32f102_bt.o(.text.BT_Soft_Reset) for BT_Soft_Reset
	Obj/mcu_initial.o(.text.BT_CONFIG) refers to Obj/FWlib_apt32f102_bt.o(.text.BT_Configure) for BT_Configure
	Obj/mcu_initial.o(.text.BT_CONFIG) refers to Obj/FWlib_apt32f102_bt.o(.text.BT_ControlSet_Configure) for BT_ControlSet_Configure
	Obj/mcu_initial.o(.text.BT_CONFIG) refers to Obj/FWlib_apt32f102_bt.o(.text.BT_Period_CMP_Write) for BT_Period_CMP_Write
	Obj/mcu_initial.o(.text.BT_CONFIG) refers to Obj/FWlib_apt32f102_bt.o(.text.BT_ConfigInterrupt_CMD) for BT_ConfigInterrupt_CMD
	FWlib_apt32f102_clkcalib.o(.text.std_clk_calib) refers to Obj/FWlib_apt32f102_bt.o(.text.BT_ConfigInterrupt_CMD) for BT_ConfigInterrupt_CMD
	Obj/mcu_initial.o(.text.BT_CONFIG) refers to Obj/FWlib_apt32f102_bt.o(.text.BT1_INT_ENABLE) for BT1_INT_ENABLE
	Obj/SYSTEM_control_rly.o(.text.Relay_Init) refers to Obj/FWlib_apt32f102_gpt.o(.text.GPT_IO_Init) for GPT_IO_Init
	Obj/SYSTEM_control_rly.o(.text.Relay_Init) refers to Obj/FWlib_apt32f102_gpt.o(.text.GPT_Configure) for GPT_Configure
	Obj/SYSTEM_control_rly.o(.text.Relay_Init) refers to Obj/FWlib_apt32f102_gpt.o(.text.GPT_WaveCtrl_Configure) for GPT_WaveCtrl_Configure
	Obj/SYSTEM_control_rly.o(.text.Relay_Init) refers to Obj/FWlib_apt32f102_gpt.o(.text.GPT_WaveLoad_Configure) for GPT_WaveLoad_Configure
	Obj/SYSTEM_control_rly.o(.text.Relay_Init) refers to Obj/FWlib_apt32f102_gpt.o(.text.GPT_WaveOut_Configure) for GPT_WaveOut_Configure
	Obj/SYSTEM_control_rly.o(.text.Relay_Init) refers to Obj/FWlib_apt32f102_gpt.o(.text.GPT_Start) for GPT_Start
	Obj/SYSTEM_control_rly.o(.text.Relay_Init) refers to Obj/FWlib_apt32f102_gpt.o(.text.GPT_Period_CMP_Write) for GPT_Period_CMP_Write
	Obj/SYSTEM_control_rly.o(.text.Relay_Init) refers to Obj/FWlib_apt32f102_gpt.o(.text.GPT_ConfigInterrupt_CMD) for GPT_ConfigInterrupt_CMD
	Obj/SYSTEM_uart.o(.text.UARTx_Init) refers to Obj/FWlib_apt32f102_uart.o(.text.UART0_DeInit) for UART0_DeInit
	Obj/SYSTEM_uart.o(.text.UARTx_Init) refers to Obj/FWlib_apt32f102_uart.o(.text.UART1_DeInit) for UART1_DeInit
	Obj/SYSTEM_uart.o(.text.UARTx_Init) refers to Obj/FWlib_apt32f102_uart.o(.text.UART2_DeInit) for UART2_DeInit
	Obj/SYSTEM_uart.o(.text.UARTx_Init) refers to Obj/FWlib_apt32f102_uart.o(.text.UART1_Int_Enable) for UART1_Int_Enable
	Obj/SYSTEM_uart.o(.text.UARTx_Init) refers to Obj/FWlib_apt32f102_uart.o(.text.UART2_Int_Enable) for UART2_Int_Enable
	Obj/SYSTEM_uart.o(.text.UARTx_Init) refers to Obj/FWlib_apt32f102_uart.o(.text.UART_IO_Init) for UART_IO_Init
	Obj/SYSTEM_uart.o(.text.UARTx_Init) refers to Obj/FWlib_apt32f102_uart.o(.text.UARTInitRxTxIntEn) for UARTInitRxTxIntEn
	Obj/SYSTEM_uart.o(.text.BUS485_Send) refers to Obj/FWlib_apt32f102_uart.o(.text.UARTTransmit) for UARTTransmit
	Obj/mcu_interrupt.o(.text.EPT0IntHandler) refers to Obj/FWlib_apt32f102_ept.o(.text.EPT_Stop) for EPT_Stop
	Obj/SYSTEM_dip_switch.o(.text.DIP_Switch_Init) refers to Obj/mcu_initial.o(.text.delay_nms) for delay_nms
	FWlib_apt32f102_clkcalib.o(.text.std_clk_calib) refers to Obj/mcu_initial.o(.text.delay_nms) for delay_nms
	Obj/SYSTEM_uart.o(.text.BUS485_Send) refers to Obj/mcu_initial.o(.text.delay_nus) for delay_nus
	Obj/mcu_initial.o(.text.APT32F102_init) refers to Obj/mcu_initial.o(.text.BT_CONFIG) for BT_CONFIG
	Obj/mcu_initial.o(.text.APT32F102_init) refers to Obj/mcu_initial.o(.text.SYSCON_CONFIG) for SYSCON_CONFIG
	Obj/main.o(.text.startup.main) refers to Obj/mcu_initial.o(.text.APT32F102_init) for APT32F102_init
	FWlib_apt32f102_tkey_c_1_17.o(.text.TK_Keymap_prog) refers to Obj/drivers_apt32f102.o(.text.__divsi3) for __divsi3
	FWlib_apt32f102_tkey_c_1_17.o(.text.TK_overflow_predict) refers to Obj/drivers_apt32f102.o(.text.__divsi3) for __divsi3
	FWlib_apt32f102_clkcalib.o(.text.std_clk_calib) refers to Obj/drivers_apt32f102.o(.text.__udivsi3) for __udivsi3
	Obj/SYSTEM_uart.o(.text.BusBusy_Task) refers to Obj/drivers_apt32f102.o(.text.__umodsi3) for __umodsi3
	Obj/mcu_initial.o(.text.APT32F102_init) refers to Obj/drivers_apt32f102_ck801.o(.text.CK_CPU_EnAllNormalIrq) for CK_CPU_EnAllNormalIrq
	Obj/SYSTEM_uart.o(.text.BUS485_Send) refers to Obj/drivers_apt32f102_ck801.o(.text.CK_CPU_EnAllNormalIrq) for CK_CPU_EnAllNormalIrq
	Obj/SYSTEM_uart.o(.text.BusIdle_Task) refers to Obj/drivers_apt32f102_ck801.o(.text.CK_CPU_EnAllNormalIrq) for CK_CPU_EnAllNormalIrq
	Obj/SYSTEM_uart.o(.text.BusBusy_Task) refers to Obj/drivers_apt32f102_ck801.o(.text.CK_CPU_EnAllNormalIrq) for CK_CPU_EnAllNormalIrq
	Obj/SYSTEM_uart.o(.text.BUS485_Send) refers to Obj/drivers_apt32f102_ck801.o(.text.CK_CPU_DisAllNormalIrq) for CK_CPU_DisAllNormalIrq
	Obj/SYSTEM_uart.o(.text.BusIdle_Task) refers to Obj/drivers_apt32f102_ck801.o(.text.CK_CPU_DisAllNormalIrq) for CK_CPU_DisAllNormalIrq
	Obj/SYSTEM_uart.o(.text.BusBusy_Task) refers to Obj/drivers_apt32f102_ck801.o(.text.CK_CPU_DisAllNormalIrq) for CK_CPU_DisAllNormalIrq
	Obj/main.o(.text.startup.main) refers to Obj/SYSTEM_uart.o(.text.Dbg_Println) for Dbg_Println
	Obj/SYSTEM_dip_switch.o(.text.DIP_Switch_Init) refers to Obj/SYSTEM_uart.o(.text.Dbg_Println) for Dbg_Println
	Obj/SYSTEM_control_rly.o(.text.BLV_VolOut_Ctrl) refers to Obj/SYSTEM_uart.o(.text.Dbg_Println) for Dbg_Println
	Obj/SYSTEM_control_rly.o(.text.BLV_RLY_Task) refers to Obj/SYSTEM_uart.o(.text.Dbg_Println) for Dbg_Println
	Obj/SYSTEM_control_rly.o(.text.BLV_RLY_RS485_Pro) refers to Obj/SYSTEM_uart.o(.text.Dbg_Println) for Dbg_Println
	Obj/mcu_initial.o(.text.APT32F102_init) refers to Obj/SYSTEM_uart.o(.text.UARTx_Init) for UARTx_Init
	Obj/mcu_interrupt.o(.text.UART1IntHandler) refers to Obj/SYSTEM_uart.o(.text.UART1_RecvINT_Processing) for UART1_RecvINT_Processing
	Obj/main.o(.text.startup.main) refers to Obj/SYSTEM_uart.o(.text.UART1_TASK) for UART1_TASK
	Obj/SYSTEM_uart.o(.text.MultSend_Task) refers to Obj/SYSTEM_uart.o(.text.BUS485_Send) for BUS485_Send
	Obj/SYSTEM_uart.o(.text.BUS485Send_Task) refers to Obj/SYSTEM_uart.o(.text.MultSend_Task) for MultSend_Task
	Obj/SYSTEM_control_rly.o(.text.BLV_A9RLY_CMD_SET_Processing) refers to Obj/SYSTEM_uart.o(.text.Set_GroupSend) for Set_GroupSend
	Obj/SYSTEM_control_rly.o(.text.BLV_A9RLY_CMD_READ_Processing) refers to Obj/SYSTEM_uart.o(.text.Set_GroupSend) for Set_GroupSend
	Obj/main.o(.text.startup.main) refers to Obj/SYSTEM_uart.o(.text.BUS485Send_Task) for BUS485Send_Task
	Obj/mcu_interrupt.o(.text.BT1IntHandler) refers to Obj/SYSTEM_uart.o(.text.BusIdle_Task) for BusIdle_Task
	Obj/mcu_interrupt.o(.text.EXI10to15IntHandler) refers to Obj/SYSTEM_uart.o(.text.BusBusy_Task) for BusBusy_Task
	Obj/SYSTEM_dip_switch.o(.text.DIP_Switch_Init) refers to Obj/SYSTEM_dip_switch.o(.text.DIP_GetSwitchState) for DIP_GetSwitchState
	Obj/SYSTEM_dip_switch.o(.text.DIP_ScanTask) refers to Obj/SYSTEM_dip_switch.o(.text.DIP_GetSwitchState) for DIP_GetSwitchState
	Obj/mcu_initial.o(.text.APT32F102_init) refers to Obj/SYSTEM_dip_switch.o(.text.DIP_Switch_Init) for DIP_Switch_Init
	Obj/main.o(.text.startup.main) refers to Obj/SYSTEM_dip_switch.o(.text.DIP_ScanTask) for DIP_ScanTask
	Obj/mcu_initial.o(.text.APT32F102_init) refers to Obj/SYSTEM_control_rly.o(.text.Relay_Init) for Relay_Init
	Obj/SYSTEM_control_rly.o(.text.BLV_A9RLY_CMD_SET_Processing) refers to Obj/SYSTEM_control_rly.o(.text.CheckSum) for CheckSum
	Obj/SYSTEM_control_rly.o(.text.BLV_A9RLY_CMD_READ_Processing) refers to Obj/SYSTEM_control_rly.o(.text.CheckSum) for CheckSum
	Obj/SYSTEM_control_rly.o(.text.BLV_RLY_RS485_Pro) refers to Obj/SYSTEM_control_rly.o(.text.CheckSum) for CheckSum
	Obj/SYSTEM_control_rly.o(.text.BLV_VolOut_Ctrl) refers to Obj/SYSTEM_control_rly.o(.text.Change_OUTV) for Change_OUTV
	Obj/SYSTEM_control_rly.o(.text.BLV_RLY_Task) refers to Obj/SYSTEM_control_rly.o(.text.BLV_VolOut_Ctrl) for BLV_VolOut_Ctrl
	Obj/SYSTEM_control_rly.o(.text.BLV_RLY_Task) refers to Obj/SYSTEM_control_rly.o(.text.BLV_RLY_Ctrl_Purpose) for BLV_RLY_Ctrl_Purpose
	Obj/SYSTEM_control_rly.o(.text.BLV_A9RLY_CMD_SET_Processing) refers to Obj/SYSTEM_control_rly.o(.text.BLV_RLY_Task) for BLV_RLY_Task
	Obj/SYSTEM_control_rly.o(.text.BLV_RLY_RS485_Pro) refers to Obj/SYSTEM_control_rly.o(.text.BLV_A9RLY_CMD_SET_Processing) for BLV_A9RLY_CMD_SET_Processing
	Obj/SYSTEM_control_rly.o(.text.BLV_RLY_RS485_Pro) refers to Obj/SYSTEM_control_rly.o(.text.BLV_A9RLY_CMD_READ_Processing) for BLV_A9RLY_CMD_READ_Processing
	FWlib_apt32f102_tkey_c_1_17.o(.text.TKEYIntHandler) refers to FWlib_apt32f102_tkey_c_1_17.o(.text.TK_Sampling_prog) for TK_Sampling_prog
	FWlib_apt32f102_tkey_c_1_17.o(.text.TK_result_prog) refers to FWlib_apt32f102_tkey_c_1_17.o(.text.get_key_number) for get_key_number
	FWlib_apt32f102_tkey_c_1_17.o(.text.CORETHandler) refers to FWlib_apt32f102_tkey_c_1_17.o(.text.TK_Scan_Start) for TK_Scan_Start
	FWlib_apt32f102_tkey_c_1_17.o(.text.CORETHandler) refers to FWlib_apt32f102_tkey_c_1_17.o(.text.TK_Keymap_prog) for TK_Keymap_prog
	FWlib_apt32f102_tkey_c_1_17.o(.text.CORETHandler) refers to FWlib_apt32f102_tkey_c_1_17.o(.text.TK_overflow_predict) for TK_overflow_predict
	FWlib_apt32f102_tkey_c_1_17.o(.text.CORETHandler) refers to FWlib_apt32f102_tkey_c_1_17.o(.text.TK_Baseline_tracking) for TK_Baseline_tracking
	FWlib_apt32f102_tkey_c_1_17.o(.text.CORETHandler) refers to FWlib_apt32f102_tkey_c_1_17.o(.text.TK_result_prog) for TK_result_prog
	Obj/mcu_initial.o(.text.SYSCON_CONFIG) refers to FWlib_apt32f102_clkcalib.o(.text.std_clk_calib) for std_clk_calib
	FWlib_apt32f102_tkey_c_1_17.o(.text.TK_overflow_predict) refers to pow.o(.text) for pow
	pow.o(.text) refers to fabs.o(.text) for fabs
	pow.o(.text) refers to scalbn.o(.text) for scalbn
	pow.o(.text) refers to sqrt.o(.text) for sqrt
	Obj/FWlib_apt32f102_gpio.o(.text.GPIO_Init) refers to _csky_case_uqi.o(.text) for ___gnu_csky_case_uqi
	Obj/FWlib_apt32f102_gpio.o(.text.GPIOA0_EXI_Init) refers to _csky_case_uqi.o(.text) for ___gnu_csky_case_uqi
	FWlib_apt32f102_tkey_c_1_17.o(.text.TK_overflow_predict) refers to _fixunsdfsi.o(.text) for __fixunsdfsi
	pow.o(.text) refers to _addsub_df.o(.text) for __adddf3
	sqrt.o(.text) refers to _addsub_df.o(.text) for __adddf3
	pow.o(.text) refers to _addsub_df.o(.text) for __subdf3
	sqrt.o(.text) refers to _addsub_df.o(.text) for __subdf3
	_fixunsdfsi.o(.text) refers to _addsub_df.o(.text) for __subdf3
	pow.o(.text) refers to _mul_df.o(.text) for __muldf3
	sqrt.o(.text) refers to _mul_df.o(.text) for __muldf3
	pow.o(.text) refers to _div_df.o(.text) for __divdf3
	sqrt.o(.text) refers to _div_df.o(.text) for __divdf3
	pow.o(.text) refers to _gt_df.o(.text) for __gtdf2
	_fixunsdfsi.o(.text) refers to _ge_df.o(.text) for __gedf2
	pow.o(.text) refers to _le_df.o(.text) for __ledf2
	pow.o(.text) refers to _si_to_df.o(.text) for __floatsidf
	_fixunsdfsi.o(.text) refers to _df_to_si.o(.text) for __fixdfsi
	FWlib_apt32f102_tkey_c_1_17.o(.text.TK_overflow_predict) refers to _usi_to_df.o(.text) for __floatunsidf
	_mul_df.o(.text) refers to _muldi3.o(.text) for __muldi3
	_si_to_df.o(.text) refers to _clzsi2.o(.text) for __clzsi2
	_usi_to_df.o(.text) refers to _clzsi2.o(.text) for __clzsi2
	_addsub_df.o(.text) refers to _pack_df.o(.text) for __pack_d
	_addsub_df.o(.text) refers to _pack_df.o(.text) for __pack_d
	_mul_df.o(.text) refers to _pack_df.o(.text) for __pack_d
	_div_df.o(.text) refers to _pack_df.o(.text) for __pack_d
	_si_to_df.o(.text) refers to _pack_df.o(.text) for __pack_d
	_usi_to_df.o(.text) refers to _pack_df.o(.text) for __pack_d
	_addsub_df.o(.text) refers to _unpack_df.o(.text) for __unpack_d
	_addsub_df.o(.text) refers to _unpack_df.o(.text) for __unpack_d
	_mul_df.o(.text) refers to _unpack_df.o(.text) for __unpack_d
	_div_df.o(.text) refers to _unpack_df.o(.text) for __unpack_d
	_gt_df.o(.text) refers to _unpack_df.o(.text) for __unpack_d
	_ge_df.o(.text) refers to _unpack_df.o(.text) for __unpack_d
	_le_df.o(.text) refers to _unpack_df.o(.text) for __unpack_d
	_df_to_si.o(.text) refers to _unpack_df.o(.text) for __unpack_d
	_gt_df.o(.text) refers to _fpcmp_parts_df.o(.text) for __fpcmp_parts_d
	_ge_df.o(.text) refers to _fpcmp_parts_df.o(.text) for __fpcmp_parts_d
	_le_df.o(.text) refers to _fpcmp_parts_df.o(.text) for __fpcmp_parts_d
	Obj/arch_mem_init.o(.text.__main) refers to memset_fast.o(.text) for memset
	Obj/SYSTEM_uart.o(.text.UARTx_Init) refers to memset_fast.o(.text) for memset
	Obj/SYSTEM_uart.o(.text.UART1_TASK) refers to memset_fast.o(.text) for memset
	Obj/SYSTEM_uart.o(.text.Set_GroupSend) refers to memset_fast.o(.text) for memset
	Obj/SYSTEM_dip_switch.o(.text.DIP_Switch_Init) refers to memset_fast.o(.text) for memset
	Obj/SYSTEM_control_rly.o(.text.Relay_Init) refers to memset_fast.o(.text) for memset
	Obj/arch_mem_init.o(.text.__main) refers to memcpy_fast.o(.text) for memcpy
	Obj/SYSTEM_uart.o(.text.UART1_TASK) refers to memcpy_fast.o(.text) for memcpy
	Obj/SYSTEM_uart.o(.text.Set_GroupSend) refers to memcpy_fast.o(.text) for memcpy
	Obj/SYSTEM_control_rly.o(.text.BLV_RLY_RS485_Pro) refers to memcpy_fast.o(.text) for memcpy


======================================================================

Removing Unused input sections from the image. 

	Removing .data(Obj/arch_crt0.o), (4 bytes).
	Removing .bss(Obj/arch_crt0.o), (0 bytes).
	Removing .text(Obj/arch_mem_init.o), (0 bytes).
	Removing .data(Obj/arch_mem_init.o), (0 bytes).
	Removing .bss(Obj/arch_mem_init.o), (0 bytes).
	Removing .text(Obj/arch_apt32f102_iostring.o), (0 bytes).
	Removing .data(Obj/arch_apt32f102_iostring.o), (0 bytes).
	Removing .bss(Obj/arch_apt32f102_iostring.o), (0 bytes).
	Removing .text.__putchar__(Obj/arch_apt32f102_iostring.o), (16 bytes).
	Removing .text.myitoa(Obj/arch_apt32f102_iostring.o), (140 bytes).
	Removing .text.my_printf(Obj/arch_apt32f102_iostring.o), (198 bytes).
	Removing .debug_info(Obj/arch_apt32f102_iostring.o), (7541 bytes).
	Removing .debug_abbrev(Obj/arch_apt32f102_iostring.o), (485 bytes).
	Removing .debug_loc(Obj/arch_apt32f102_iostring.o), (653 bytes).
	Removing .debug_aranges(Obj/arch_apt32f102_iostring.o), (48 bytes).
	Removing .debug_ranges(Obj/arch_apt32f102_iostring.o), (32 bytes).
	Removing .debug_line(Obj/arch_apt32f102_iostring.o), (487 bytes).
	Removing .debug_str(Obj/arch_apt32f102_iostring.o), (2911 bytes).
	Removing .comment(Obj/arch_apt32f102_iostring.o), (67 bytes).
	Removing .debug_frame(Obj/arch_apt32f102_iostring.o), (120 bytes).
	Removing .csky.attributes(Obj/arch_apt32f102_iostring.o), (32 bytes).
	Removing .text(Obj/FWlib_apt32f102_syscon.o), (0 bytes).
	Removing .data(Obj/FWlib_apt32f102_syscon.o), (0 bytes).
	Removing .bss(Obj/FWlib_apt32f102_syscon.o), (0 bytes).
	Removing .text.EMOSC_OSTR_Config(Obj/FWlib_apt32f102_syscon.o), (28 bytes).
	Removing .text.SystemCLK_Clear(Obj/FWlib_apt32f102_syscon.o), (24 bytes).
	Removing .text.SYSCON_IMOSC_SELECTE(Obj/FWlib_apt32f102_syscon.o), (20 bytes).
	Removing .text.LVD_Int_Disable(Obj/FWlib_apt32f102_syscon.o), (16 bytes).
	Removing .text.IWDT_Int_Disable(Obj/FWlib_apt32f102_syscon.o), (16 bytes).
	Removing .text.Read_Reset_Status(Obj/FWlib_apt32f102_syscon.o), (24 bytes).
	Removing .text.PCLK_goto_idle_mode(Obj/FWlib_apt32f102_syscon.o), (6 bytes).
	Removing .text.PCLK_goto_deepsleep_mode(Obj/FWlib_apt32f102_syscon.o), (20 bytes).
	Removing .text.EXI0_Int_Enable(Obj/FWlib_apt32f102_syscon.o), (12 bytes).
	Removing .text.EXI0_Int_Disable(Obj/FWlib_apt32f102_syscon.o), (12 bytes).
	Removing .text.EXI1_Int_Enable(Obj/FWlib_apt32f102_syscon.o), (16 bytes).
	Removing .text.EXI1_Int_Disable(Obj/FWlib_apt32f102_syscon.o), (16 bytes).
	Removing .text.EXI2_Int_Enable(Obj/FWlib_apt32f102_syscon.o), (16 bytes).
	Removing .text.EXI2_Int_Disable(Obj/FWlib_apt32f102_syscon.o), (16 bytes).
	Removing .text.EXI3_Int_Enable(Obj/FWlib_apt32f102_syscon.o), (16 bytes).
	Removing .text.EXI3_Int_Disable(Obj/FWlib_apt32f102_syscon.o), (16 bytes).
	Removing .text.EXI4_Int_Disable(Obj/FWlib_apt32f102_syscon.o), (16 bytes).
	Removing .text.EXI0_WakeUp_Enable(Obj/FWlib_apt32f102_syscon.o), (12 bytes).
	Removing .text.EXI0_WakeUp_Disable(Obj/FWlib_apt32f102_syscon.o), (12 bytes).
	Removing .text.EXI1_WakeUp_Enable(Obj/FWlib_apt32f102_syscon.o), (16 bytes).
	Removing .text.EXI1_WakeUp_Disable(Obj/FWlib_apt32f102_syscon.o), (16 bytes).
	Removing .text.EXI2_WakeUp_Enable(Obj/FWlib_apt32f102_syscon.o), (16 bytes).
	Removing .text.EXI2_WakeUp_Disable(Obj/FWlib_apt32f102_syscon.o), (16 bytes).
	Removing .text.EXI3_WakeUp_Enable(Obj/FWlib_apt32f102_syscon.o), (16 bytes).
	Removing .text.EXI3_WakeUp_Disable(Obj/FWlib_apt32f102_syscon.o), (16 bytes).
	Removing .text.EXI4_WakeUp_Enable(Obj/FWlib_apt32f102_syscon.o), (16 bytes).
	Removing .text.EXI4_WakeUp_Disable(Obj/FWlib_apt32f102_syscon.o), (16 bytes).
	Removing .text.SYSCON_WakeUp_Enable(Obj/FWlib_apt32f102_syscon.o), (12 bytes).
	Removing .text.SYSCON_CLO_CONFIG(Obj/FWlib_apt32f102_syscon.o), (52 bytes).
	Removing .text.SYSCON_CLO_SRC_SET(Obj/FWlib_apt32f102_syscon.o), (32 bytes).
	Removing .text.SYSCON_WakeUp_Disable(Obj/FWlib_apt32f102_syscon.o), (12 bytes).
	Removing .text.SYSCON_Read_CINF0(Obj/FWlib_apt32f102_syscon.o), (16 bytes).
	Removing .text.SYSCON_Read_CINF1(Obj/FWlib_apt32f102_syscon.o), (16 bytes).
	Removing .text.SYSCON_Software_Reset(Obj/FWlib_apt32f102_syscon.o), (20 bytes).
	Removing .text.GPIO_Remap(Obj/FWlib_apt32f102_syscon.o), (652 bytes).
	Removing .text(Obj/FWlib_apt32f102_gpio.o), (0 bytes).
	Removing .data(Obj/FWlib_apt32f102_gpio.o), (0 bytes).
	Removing .bss(Obj/FWlib_apt32f102_gpio.o), (0 bytes).
	Removing .text.GPIO_DeInit(Obj/FWlib_apt32f102_gpio.o), (100 bytes).
	Removing .text.GPIO_Init2(Obj/FWlib_apt32f102_gpio.o), (16 bytes).
	Removing .text.GPIO_InPutOutPut_Disable(Obj/FWlib_apt32f102_gpio.o), (164 bytes).
	Removing .text.GPIO_MODE_Init(Obj/FWlib_apt32f102_gpio.o), (34 bytes).
	Removing .text.GPIO_PullLow_Init(Obj/FWlib_apt32f102_gpio.o), (20 bytes).
	Removing .text.GPIO_PullHighLow_DIS(Obj/FWlib_apt32f102_gpio.o), (14 bytes).
	Removing .text.GPIO_OpenDrain_EN(Obj/FWlib_apt32f102_gpio.o), (12 bytes).
	Removing .text.GPIO_OpenDrain_DIS(Obj/FWlib_apt32f102_gpio.o), (14 bytes).
	Removing .text.GPIO_TTL_COSM_Selecte(Obj/FWlib_apt32f102_gpio.o), (72 bytes).
	Removing .text.GPIO_DriveStrength_DIS(Obj/FWlib_apt32f102_gpio.o), (16 bytes).
	Removing .text.GPIOB0_EXI_Init(Obj/FWlib_apt32f102_gpio.o), (108 bytes).
	Removing .text.GPIO_EXI_EN(Obj/FWlib_apt32f102_gpio.o), (12 bytes).
	Removing .text.GPIO_Set_Value(Obj/FWlib_apt32f102_gpio.o), (22 bytes).
	Removing .text.GPIO_Read_Output(Obj/FWlib_apt32f102_gpio.o), (16 bytes).
	Removing .text(Obj/FWlib_apt32f102_lpt.o), (0 bytes).
	Removing .data(Obj/FWlib_apt32f102_lpt.o), (0 bytes).
	Removing .bss(Obj/FWlib_apt32f102_lpt.o), (0 bytes).
	Removing .text.LPT_DeInit(Obj/FWlib_apt32f102_lpt.o), (60 bytes).
	Removing .text.LPT_IO_Init(Obj/FWlib_apt32f102_lpt.o), (72 bytes).
	Removing .text.LPT_Configure(Obj/FWlib_apt32f102_lpt.o), (44 bytes).
	Removing .text.LPT_Debug_Mode(Obj/FWlib_apt32f102_lpt.o), (24 bytes).
	Removing .text.LPT_Period_CMP_Write(Obj/FWlib_apt32f102_lpt.o), (16 bytes).
	Removing .text.LPT_CNT_Write(Obj/FWlib_apt32f102_lpt.o), (12 bytes).
	Removing .text.LPT_PRDR_Read(Obj/FWlib_apt32f102_lpt.o), (16 bytes).
	Removing .text.LPT_CMP_Read(Obj/FWlib_apt32f102_lpt.o), (16 bytes).
	Removing .text.LPT_CNT_Read(Obj/FWlib_apt32f102_lpt.o), (16 bytes).
	Removing .text.LPT_ControlSet_Configure(Obj/FWlib_apt32f102_lpt.o), (40 bytes).
	Removing .text.LPT_SyncSet_Configure(Obj/FWlib_apt32f102_lpt.o), (24 bytes).
	Removing .text.LPT_Trigger_Configure(Obj/FWlib_apt32f102_lpt.o), (72 bytes).
	Removing .text.LPT_Trigger_EVPS(Obj/FWlib_apt32f102_lpt.o), (20 bytes).
	Removing .text.LPT_Trigger_Cnt(Obj/FWlib_apt32f102_lpt.o), (20 bytes).
	Removing .text.LPT_Soft_Trigger(Obj/FWlib_apt32f102_lpt.o), (16 bytes).
	Removing .text.LPT_Start(Obj/FWlib_apt32f102_lpt.o), (16 bytes).
	Removing .text.LPT_Stop(Obj/FWlib_apt32f102_lpt.o), (16 bytes).
	Removing .text.LPT_REARM_Write(Obj/FWlib_apt32f102_lpt.o), (16 bytes).
	Removing .text.LPT_REARM_Read(Obj/FWlib_apt32f102_lpt.o), (20 bytes).
	Removing .text.LPT_ConfigInterrupt_CMD(Obj/FWlib_apt32f102_lpt.o), (28 bytes).
	Removing .text.LPT_INT_ENABLE(Obj/FWlib_apt32f102_lpt.o), (16 bytes).
	Removing .text.LPT_INT_DISABLE(Obj/FWlib_apt32f102_lpt.o), (16 bytes).
	Removing .text(Obj/FWlib_apt32f102_crc.o), (0 bytes).
	Removing .data(Obj/FWlib_apt32f102_crc.o), (0 bytes).
	Removing .bss(Obj/FWlib_apt32f102_crc.o), (0 bytes).
	Removing .text.CRC_CMD(Obj/FWlib_apt32f102_crc.o), (24 bytes).
	Removing .text.CRC_Soft_Reset(Obj/FWlib_apt32f102_crc.o), (16 bytes).
	Removing .text.CRC_Configure(Obj/FWlib_apt32f102_crc.o), (36 bytes).
	Removing .text.CRC_Seed_Write(Obj/FWlib_apt32f102_crc.o), (12 bytes).
	Removing .text.CRC_Seed_Read(Obj/FWlib_apt32f102_crc.o), (12 bytes).
	Removing .text.CRC_Datain(Obj/FWlib_apt32f102_crc.o), (12 bytes).
	Removing .text.CRC_Result_Read(Obj/FWlib_apt32f102_crc.o), (12 bytes).
	Removing .text.Chip_CRC_CRC32(Obj/FWlib_apt32f102_crc.o), (28 bytes).
	Removing .text.Chip_CRC_CRC16(Obj/FWlib_apt32f102_crc.o), (52 bytes).
	Removing .text.Chip_CRC_CRC8(Obj/FWlib_apt32f102_crc.o), (44 bytes).
	Removing .debug_info(Obj/FWlib_apt32f102_crc.o), (7732 bytes).
	Removing .debug_abbrev(Obj/FWlib_apt32f102_crc.o), (592 bytes).
	Removing .debug_loc(Obj/FWlib_apt32f102_crc.o), (358 bytes).
	Removing .debug_aranges(Obj/FWlib_apt32f102_crc.o), (104 bytes).
	Removing .debug_ranges(Obj/FWlib_apt32f102_crc.o), (112 bytes).
	Removing .debug_line(Obj/FWlib_apt32f102_crc.o), (350 bytes).
	Removing .debug_str(Obj/FWlib_apt32f102_crc.o), (3105 bytes).
	Removing .comment(Obj/FWlib_apt32f102_crc.o), (67 bytes).
	Removing .debug_frame(Obj/FWlib_apt32f102_crc.o), (204 bytes).
	Removing .csky.attributes(Obj/FWlib_apt32f102_crc.o), (32 bytes).
	Removing .text(Obj/FWlib_apt32f102_wwdt.o), (0 bytes).
	Removing .data(Obj/FWlib_apt32f102_wwdt.o), (0 bytes).
	Removing .bss(Obj/FWlib_apt32f102_wwdt.o), (0 bytes).
	Removing .text.WWDT_DeInit(Obj/FWlib_apt32f102_wwdt.o), (28 bytes).
	Removing .text.WWDT_CONFIG(Obj/FWlib_apt32f102_wwdt.o), (24 bytes).
	Removing .text.WWDT_CMD(Obj/FWlib_apt32f102_wwdt.o), (24 bytes).
	Removing .text.WWDT_Int_Config(Obj/FWlib_apt32f102_wwdt.o), (52 bytes).
	Removing .text(Obj/FWlib_apt32f102_countera.o), (0 bytes).
	Removing .data(Obj/FWlib_apt32f102_countera.o), (0 bytes).
	Removing .bss(Obj/FWlib_apt32f102_countera.o), (0 bytes).
	Removing .text.COUNT_DeInit(Obj/FWlib_apt32f102_countera.o), (20 bytes).
	Removing .text.COUNTA_Int_Enable(Obj/FWlib_apt32f102_countera.o), (16 bytes).
	Removing .text.COUNTA_Int_Disable(Obj/FWlib_apt32f102_countera.o), (16 bytes).
	Removing .text.COUNTA_Wakeup_Enable(Obj/FWlib_apt32f102_countera.o), (16 bytes).
	Removing .text.COUNTA_Wakeup_Disable(Obj/FWlib_apt32f102_countera.o), (16 bytes).
	Removing .text.COUNTA_Init(Obj/FWlib_apt32f102_countera.o), (60 bytes).
	Removing .text.COUNTA_Config(Obj/FWlib_apt32f102_countera.o), (32 bytes).
	Removing .text.COUNTA_Start(Obj/FWlib_apt32f102_countera.o), (20 bytes).
	Removing .text.COUNTA_Stop(Obj/FWlib_apt32f102_countera.o), (16 bytes).
	Removing .text.COUNTA_Data_Update(Obj/FWlib_apt32f102_countera.o), (20 bytes).
	Removing .text.COUNTA_IO_Init(Obj/FWlib_apt32f102_countera.o), (80 bytes).
	Removing .debug_info(Obj/FWlib_apt32f102_countera.o), (7799 bytes).
	Removing .debug_abbrev(Obj/FWlib_apt32f102_countera.o), (381 bytes).
	Removing .debug_loc(Obj/FWlib_apt32f102_countera.o), (336 bytes).
	Removing .debug_aranges(Obj/FWlib_apt32f102_countera.o), (112 bytes).
	Removing .debug_ranges(Obj/FWlib_apt32f102_countera.o), (96 bytes).
	Removing .debug_line(Obj/FWlib_apt32f102_countera.o), (350 bytes).
	Removing .debug_str(Obj/FWlib_apt32f102_countera.o), (3422 bytes).
	Removing .comment(Obj/FWlib_apt32f102_countera.o), (67 bytes).
	Removing .debug_frame(Obj/FWlib_apt32f102_countera.o), (224 bytes).
	Removing .csky.attributes(Obj/FWlib_apt32f102_countera.o), (32 bytes).
	Removing .text(Obj/FWlib_apt32f102_et.o), (0 bytes).
	Removing .data(Obj/FWlib_apt32f102_et.o), (0 bytes).
	Removing .bss(Obj/FWlib_apt32f102_et.o), (0 bytes).
	Removing .text.ET_DeInit(Obj/FWlib_apt32f102_et.o), (40 bytes).
	Removing .text.ET_ENABLE(Obj/FWlib_apt32f102_et.o), (16 bytes).
	Removing .text.ET_DISABLE(Obj/FWlib_apt32f102_et.o), (16 bytes).
	Removing .text.ET_SWTRG_CMD(Obj/FWlib_apt32f102_et.o), (28 bytes).
	Removing .text.ET_CH0_SRCSEL(Obj/FWlib_apt32f102_et.o), (108 bytes).
	Removing .text.ET_CH0_CONTROL(Obj/FWlib_apt32f102_et.o), (40 bytes).
	Removing .text.ET_CH1_SRCSEL(Obj/FWlib_apt32f102_et.o), (108 bytes).
	Removing .text.ET_CH1_CONTROL(Obj/FWlib_apt32f102_et.o), (40 bytes).
	Removing .text.ET_CH2_SRCSEL(Obj/FWlib_apt32f102_et.o), (108 bytes).
	Removing .text.ET_CH2_CONTROL(Obj/FWlib_apt32f102_et.o), (40 bytes).
	Removing .text.ET_CHx_CONTROL(Obj/FWlib_apt32f102_et.o), (276 bytes).
	Removing .debug_info(Obj/FWlib_apt32f102_et.o), (7781 bytes).
	Removing .debug_abbrev(Obj/FWlib_apt32f102_et.o), (410 bytes).
	Removing .debug_loc(Obj/FWlib_apt32f102_et.o), (1318 bytes).
	Removing .debug_aranges(Obj/FWlib_apt32f102_et.o), (112 bytes).
	Removing .debug_ranges(Obj/FWlib_apt32f102_et.o), (96 bytes).
	Removing .debug_line(Obj/FWlib_apt32f102_et.o), (463 bytes).
	Removing .debug_str(Obj/FWlib_apt32f102_et.o), (3167 bytes).
	Removing .comment(Obj/FWlib_apt32f102_et.o), (67 bytes).
	Removing .debug_frame(Obj/FWlib_apt32f102_et.o), (204 bytes).
	Removing .csky.attributes(Obj/FWlib_apt32f102_et.o), (32 bytes).
	Removing .text(Obj/FWlib_apt32f102_bt.o), (0 bytes).
	Removing .data(Obj/FWlib_apt32f102_bt.o), (0 bytes).
	Removing .bss(Obj/FWlib_apt32f102_bt.o), (0 bytes).
	Removing .text.BT_IO_Init(Obj/FWlib_apt32f102_bt.o), (332 bytes).
	Removing .text.BT_Stop(Obj/FWlib_apt32f102_bt.o), (8 bytes).
	Removing .text.BT_Stop_High(Obj/FWlib_apt32f102_bt.o), (14 bytes).
	Removing .text.BT_Stop_Low(Obj/FWlib_apt32f102_bt.o), (14 bytes).
	Removing .text.BT_CNT_Write(Obj/FWlib_apt32f102_bt.o), (4 bytes).
	Removing .text.BT_PRDR_Read(Obj/FWlib_apt32f102_bt.o), (6 bytes).
	Removing .text.BT_CMP_Read(Obj/FWlib_apt32f102_bt.o), (6 bytes).
	Removing .text.BT_CNT_Read(Obj/FWlib_apt32f102_bt.o), (6 bytes).
	Removing .text.BT_Trigger_Configure(Obj/FWlib_apt32f102_bt.o), (10 bytes).
	Removing .text.BT_Soft_Tigger(Obj/FWlib_apt32f102_bt.o), (6 bytes).
	Removing .text.BT0_INT_ENABLE(Obj/FWlib_apt32f102_bt.o), (16 bytes).
	Removing .text.BT0_INT_DISABLE(Obj/FWlib_apt32f102_bt.o), (16 bytes).
	Removing .text.BT1_INT_DISABLE(Obj/FWlib_apt32f102_bt.o), (16 bytes).
	Removing .text(Obj/FWlib_apt32f102_gpt.o), (0 bytes).
	Removing .data(Obj/FWlib_apt32f102_gpt.o), (0 bytes).
	Removing .bss(Obj/FWlib_apt32f102_gpt.o), (0 bytes).
	Removing .text.GPT_DeInit(Obj/FWlib_apt32f102_gpt.o), (96 bytes).
	Removing .text.GPT_Capture_Config(Obj/FWlib_apt32f102_gpt.o), (68 bytes).
	Removing .text.GPT_SyncSet_Configure(Obj/FWlib_apt32f102_gpt.o), (36 bytes).
	Removing .text.GPT_Trigger_Configure(Obj/FWlib_apt32f102_gpt.o), (44 bytes).
	Removing .text.GPT_EVTRG_Configure(Obj/FWlib_apt32f102_gpt.o), (92 bytes).
	Removing .text.GPT_OneceForce_Out(Obj/FWlib_apt32f102_gpt.o), (32 bytes).
	Removing .text.GPT_Force_Out(Obj/FWlib_apt32f102_gpt.o), (16 bytes).
	Removing .text.GPT_CmpLoad_Configure(Obj/FWlib_apt32f102_gpt.o), (20 bytes).
	Removing .text.GPT_Debug_Mode(Obj/FWlib_apt32f102_gpt.o), (24 bytes).
	Removing .text.GPT_Stop(Obj/FWlib_apt32f102_gpt.o), (16 bytes).
	Removing .text.GPT_Soft_Reset(Obj/FWlib_apt32f102_gpt.o), (20 bytes).
	Removing .text.GPT_Cap_Rearm(Obj/FWlib_apt32f102_gpt.o), (16 bytes).
	Removing .text.GPT_Mode_CMD(Obj/FWlib_apt32f102_gpt.o), (16 bytes).
	Removing .text.GPT_REARM_Write(Obj/FWlib_apt32f102_gpt.o), (16 bytes).
	Removing .text.GPT_REARM_Read(Obj/FWlib_apt32f102_gpt.o), (20 bytes).
	Removing .text.GPT_PRDR_Read(Obj/FWlib_apt32f102_gpt.o), (16 bytes).
	Removing .text.GPT_CMPA_Read(Obj/FWlib_apt32f102_gpt.o), (16 bytes).
	Removing .text.GPT_CMPB_Read(Obj/FWlib_apt32f102_gpt.o), (16 bytes).
	Removing .text.GPT_CNT_Read(Obj/FWlib_apt32f102_gpt.o), (16 bytes).
	Removing .text.GPT_INT_ENABLE(Obj/FWlib_apt32f102_gpt.o), (16 bytes).
	Removing .text.GPT_INT_DISABLE(Obj/FWlib_apt32f102_gpt.o), (16 bytes).
	Removing .text(Obj/FWlib_apt32f102_sio.o), (0 bytes).
	Removing .data(Obj/FWlib_apt32f102_sio.o), (0 bytes).
	Removing .bss(Obj/FWlib_apt32f102_sio.o), (0 bytes).
	Removing .text.SIO_DeInit(Obj/FWlib_apt32f102_sio.o), (32 bytes).
	Removing .text.SIO_IO_Init(Obj/FWlib_apt32f102_sio.o), (96 bytes).
	Removing .text.SIO_TX_Init(Obj/FWlib_apt32f102_sio.o), (16 bytes).
	Removing .text.SIO_TX_Configure(Obj/FWlib_apt32f102_sio.o), (80 bytes).
	Removing .text.SIO_TXBUF_Set(Obj/FWlib_apt32f102_sio.o), (156 bytes).
	Removing .text.SIO_RX_Init(Obj/FWlib_apt32f102_sio.o), (20 bytes).
	Removing .text.SIO_RX_Configure0(Obj/FWlib_apt32f102_sio.o), (96 bytes).
	Removing .text.SIO_RX_Configure1(Obj/FWlib_apt32f102_sio.o), (32 bytes).
	Removing .text.SIO_ConfigInterrupt_CMD(Obj/FWlib_apt32f102_sio.o), (28 bytes).
	Removing .text.SIO_INT_ENABLE(Obj/FWlib_apt32f102_sio.o), (16 bytes).
	Removing .text.SIO_INT_DISABLE(Obj/FWlib_apt32f102_sio.o), (16 bytes).
	Removing .debug_info(Obj/FWlib_apt32f102_sio.o), (8669 bytes).
	Removing .debug_abbrev(Obj/FWlib_apt32f102_sio.o), (405 bytes).
	Removing .debug_loc(Obj/FWlib_apt32f102_sio.o), (1996 bytes).
	Removing .debug_aranges(Obj/FWlib_apt32f102_sio.o), (112 bytes).
	Removing .debug_ranges(Obj/FWlib_apt32f102_sio.o), (96 bytes).
	Removing .debug_line(Obj/FWlib_apt32f102_sio.o), (391 bytes).
	Removing .debug_str(Obj/FWlib_apt32f102_sio.o), (4135 bytes).
	Removing .comment(Obj/FWlib_apt32f102_sio.o), (67 bytes).
	Removing .debug_frame(Obj/FWlib_apt32f102_sio.o), (260 bytes).
	Removing .csky.attributes(Obj/FWlib_apt32f102_sio.o), (32 bytes).
	Removing .text(Obj/FWlib_apt32f102_spi.o), (0 bytes).
	Removing .data(Obj/FWlib_apt32f102_spi.o), (0 bytes).
	Removing .bss(Obj/FWlib_apt32f102_spi.o), (0 bytes).
	Removing .text.SPI_DeInit(Obj/FWlib_apt32f102_spi.o), (32 bytes).
	Removing .text.SPI_NSS_IO_Init(Obj/FWlib_apt32f102_spi.o), (52 bytes).
	Removing .text.SPI_Master_Init(Obj/FWlib_apt32f102_spi.o), (176 bytes).
	Removing .text.SPI_Slave_Init(Obj/FWlib_apt32f102_spi.o), (156 bytes).
	Removing .text.SPI_WRITE_BYTE(Obj/FWlib_apt32f102_spi.o), (32 bytes).
	Removing .text.SPI_READ_BYTE(Obj/FWlib_apt32f102_spi.o), (100 bytes).
	Removing .text.SPI_ConfigInterrupt_CMD(Obj/FWlib_apt32f102_spi.o), (28 bytes).
	Removing .text.SPI_Int_Enable(Obj/FWlib_apt32f102_spi.o), (16 bytes).
	Removing .text.SPI_Int_Disable(Obj/FWlib_apt32f102_spi.o), (16 bytes).
	Removing .text.SPI_Wakeup_Enable(Obj/FWlib_apt32f102_spi.o), (16 bytes).
	Removing .text.SPI_Wakeup_Disable(Obj/FWlib_apt32f102_spi.o), (16 bytes).
	Removing .debug_info(Obj/FWlib_apt32f102_spi.o), (7854 bytes).
	Removing .debug_abbrev(Obj/FWlib_apt32f102_spi.o), (402 bytes).
	Removing .debug_loc(Obj/FWlib_apt32f102_spi.o), (641 bytes).
	Removing .debug_aranges(Obj/FWlib_apt32f102_spi.o), (112 bytes).
	Removing .debug_ranges(Obj/FWlib_apt32f102_spi.o), (96 bytes).
	Removing .debug_line(Obj/FWlib_apt32f102_spi.o), (407 bytes).
	Removing .debug_str(Obj/FWlib_apt32f102_spi.o), (3538 bytes).
	Removing .comment(Obj/FWlib_apt32f102_spi.o), (67 bytes).
	Removing .debug_frame(Obj/FWlib_apt32f102_spi.o), (240 bytes).
	Removing .csky.attributes(Obj/FWlib_apt32f102_spi.o), (32 bytes).
	Removing .text(Obj/FWlib_apt32f102_uart.o), (0 bytes).
	Removing .data(Obj/FWlib_apt32f102_uart.o), (0 bytes).
	Removing .bss(Obj/FWlib_apt32f102_uart.o), (2 bytes).
	Removing .text.UART0_Int_Enable(Obj/FWlib_apt32f102_uart.o), (28 bytes).
	Removing .text.UART0_Int_Disable(Obj/FWlib_apt32f102_uart.o), (16 bytes).
	Removing .text.UART1_Int_Disable(Obj/FWlib_apt32f102_uart.o), (16 bytes).
	Removing .text.UART2_Int_Disable(Obj/FWlib_apt32f102_uart.o), (16 bytes).
	Removing .text.UART0_WakeUp_Enable(Obj/FWlib_apt32f102_uart.o), (16 bytes).
	Removing .text.UART0_WakeUp_Disable(Obj/FWlib_apt32f102_uart.o), (16 bytes).
	Removing .text.UART1_WakeUp_Enable(Obj/FWlib_apt32f102_uart.o), (16 bytes).
	Removing .text.UART1_WakeUp_Disable(Obj/FWlib_apt32f102_uart.o), (16 bytes).
	Removing .text.UART2_WakeUp_Enable(Obj/FWlib_apt32f102_uart.o), (16 bytes).
	Removing .text.UART2_WakeUp_Disable(Obj/FWlib_apt32f102_uart.o), (16 bytes).
	Removing .text.UARTInit(Obj/FWlib_apt32f102_uart.o), (16 bytes).
	Removing .text.UARTInitRxIntEn(Obj/FWlib_apt32f102_uart.o), (10 bytes).
	Removing .text.UARTClose(Obj/FWlib_apt32f102_uart.o), (6 bytes).
	Removing .text.UARTTxByte(Obj/FWlib_apt32f102_uart.o), (14 bytes).
	Removing .text.UARTTTransmit_data_set(Obj/FWlib_apt32f102_uart.o), (44 bytes).
	Removing .text.UARTTransmit_INT_Send(Obj/FWlib_apt32f102_uart.o), (72 bytes).
	Removing .text.UARTRxByte(Obj/FWlib_apt32f102_uart.o), (22 bytes).
	Removing .text.UART_ReturnRxByte(Obj/FWlib_apt32f102_uart.o), (24 bytes).
	Removing .text.UARTReceive(Obj/FWlib_apt32f102_uart.o), (56 bytes).
	Removing COMMON(Obj/FWlib_apt32f102_uart.o), (36 bytes).
	Removing .text(Obj/FWlib_apt32f102_i2c.o), (0 bytes).
	Removing .data(Obj/FWlib_apt32f102_i2c.o), (0 bytes).
	Removing .bss(Obj/FWlib_apt32f102_i2c.o), (6 bytes).
	Removing .text.I2C_DeInit(Obj/FWlib_apt32f102_i2c.o), (24 bytes).
	Removing .text.I2C_Master_CONFIG(Obj/FWlib_apt32f102_i2c.o), (320 bytes).
	Removing .text.I2C_Slave_CONFIG(Obj/FWlib_apt32f102_i2c.o), (332 bytes).
	Removing .text.I2C_SDA_TSETUP_THOLD_CONFIG(Obj/FWlib_apt32f102_i2c.o), (20 bytes).
	Removing .text.I2C_ConfigInterrupt_CMD(Obj/FWlib_apt32f102_i2c.o), (28 bytes).
	Removing .text.I2C_FIFO_TriggerData(Obj/FWlib_apt32f102_i2c.o), (16 bytes).
	Removing .text.I2C_Stop(Obj/FWlib_apt32f102_i2c.o), (16 bytes).
	Removing .text.I2C_Enable(Obj/FWlib_apt32f102_i2c.o), (28 bytes).
	Removing .text.I2C_Disable(Obj/FWlib_apt32f102_i2c.o), (28 bytes).
	Removing .text.I2C_Abort_EN(Obj/FWlib_apt32f102_i2c.o), (16 bytes).
	Removing .text.I2C_Abort_Status(Obj/FWlib_apt32f102_i2c.o), (20 bytes).
	Removing .text.I2C_SDA_Recover_EN(Obj/FWlib_apt32f102_i2c.o), (16 bytes).
	Removing .text.I2C_SDA_Recover_DIS(Obj/FWlib_apt32f102_i2c.o), (16 bytes).
	Removing .text.I2C_Int_Enable(Obj/FWlib_apt32f102_i2c.o), (16 bytes).
	Removing .text.I2C_Int_Disable(Obj/FWlib_apt32f102_i2c.o), (16 bytes).
	Removing .text.I2C_WRITE_Byte(Obj/FWlib_apt32f102_i2c.o), (112 bytes).
	Removing .text.I2C_WRITE_nByte(Obj/FWlib_apt32f102_i2c.o), (160 bytes).
	Removing .text.I2C_READ_Byte(Obj/FWlib_apt32f102_i2c.o), (100 bytes).
	Removing .text.I2C_READ_nByte(Obj/FWlib_apt32f102_i2c.o), (160 bytes).
	Removing .text.I2C_Slave_Receive(Obj/FWlib_apt32f102_i2c.o), (384 bytes).
	Removing .debug_info(Obj/FWlib_apt32f102_i2c.o), (8426 bytes).
	Removing .debug_abbrev(Obj/FWlib_apt32f102_i2c.o), (576 bytes).
	Removing .debug_loc(Obj/FWlib_apt32f102_i2c.o), (1150 bytes).
	Removing .debug_aranges(Obj/FWlib_apt32f102_i2c.o), (184 bytes).
	Removing .debug_ranges(Obj/FWlib_apt32f102_i2c.o), (168 bytes).
	Removing .debug_line(Obj/FWlib_apt32f102_i2c.o), (847 bytes).
	Removing .debug_str(Obj/FWlib_apt32f102_i2c.o), (3654 bytes).
	Removing .comment(Obj/FWlib_apt32f102_i2c.o), (67 bytes).
	Removing .debug_frame(Obj/FWlib_apt32f102_i2c.o), (452 bytes).
	Removing .csky.attributes(Obj/FWlib_apt32f102_i2c.o), (32 bytes).
	Removing COMMON(Obj/FWlib_apt32f102_i2c.o), (70 bytes).
	Removing .text(Obj/FWlib_apt32f102_ept.o), (0 bytes).
	Removing .data(Obj/FWlib_apt32f102_ept.o), (0 bytes).
	Removing .bss(Obj/FWlib_apt32f102_ept.o), (0 bytes).
	Removing .text.EPT_Software_Prg(Obj/FWlib_apt32f102_ept.o), (32 bytes).
	Removing .text.EPT_Start(Obj/FWlib_apt32f102_ept.o), (40 bytes).
	Removing .text.EPT_IO_SET(Obj/FWlib_apt32f102_ept.o), (568 bytes).
	Removing .text.EPT_PWM_Config(Obj/FWlib_apt32f102_ept.o), (56 bytes).
	Removing .text.EPT_CG_gate_Config(Obj/FWlib_apt32f102_ept.o), (116 bytes).
	Removing .text.EPT_Capture_Config(Obj/FWlib_apt32f102_ept.o), (104 bytes).
	Removing .text.EPT_SYNCR_Config(Obj/FWlib_apt32f102_ept.o), (52 bytes).
	Removing .text.EPT_CPCR_Config(Obj/FWlib_apt32f102_ept.o), (80 bytes).
	Removing .text.EPT_DBCR_Config(Obj/FWlib_apt32f102_ept.o), (96 bytes).
	Removing .text.EPT_DB_CLK_Config(Obj/FWlib_apt32f102_ept.o), (16 bytes).
	Removing .text.EPT_PWMX_Output_Control(Obj/FWlib_apt32f102_ept.o), (216 bytes).
	Removing .text.EPT_Tevent_Selecte(Obj/FWlib_apt32f102_ept.o), (16 bytes).
	Removing .text.EPT_PHSEN_Config(Obj/FWlib_apt32f102_ept.o), (24 bytes).
	Removing .text.EPT_PRDR_CMPA_CMPB_CMPC_CMPD_Config(Obj/FWlib_apt32f102_ept.o), (28 bytes).
	Removing .text.EPT_SYNCR_RearmClr(Obj/FWlib_apt32f102_ept.o), (40 bytes).
	Removing .text.EPT_Caputure_Rearm(Obj/FWlib_apt32f102_ept.o), (20 bytes).
	Removing .text.EPT_Globle_Eventload_Config(Obj/FWlib_apt32f102_ept.o), (24 bytes).
	Removing .text.EPT_Globle_SwLoad_CMD(Obj/FWlib_apt32f102_ept.o), (28 bytes).
	Removing .text.EPT_PRDR_EventLoad_Config(Obj/FWlib_apt32f102_ept.o), (28 bytes).
	Removing .text.EPT_CMP_EventLoad_Config(Obj/FWlib_apt32f102_ept.o), (68 bytes).
	Removing .text.EPT_AQCR_Eventload_Config(Obj/FWlib_apt32f102_ept.o), (72 bytes).
	Removing .text.EPT_DB_Eventload_Config(Obj/FWlib_apt32f102_ept.o), (72 bytes).
	Removing .text.EPT_TRGSRCX_Config(Obj/FWlib_apt32f102_ept.o), (136 bytes).
	Removing .text.EPT_TRGSRCX_SWFTRG(Obj/FWlib_apt32f102_ept.o), (72 bytes).
	Removing .text.EPT_Int_Enable(Obj/FWlib_apt32f102_ept.o), (20 bytes).
	Removing .text.EPT_Int_Disable(Obj/FWlib_apt32f102_ept.o), (20 bytes).
	Removing .text.EPT_EMInt_Enable(Obj/FWlib_apt32f102_ept.o), (20 bytes).
	Removing .text.EPT_EMInt_Disable(Obj/FWlib_apt32f102_ept.o), (20 bytes).
	Removing .text.EPT_Vector_Int_Enable(Obj/FWlib_apt32f102_ept.o), (12 bytes).
	Removing .text.EPT_Vector_Int_Disable(Obj/FWlib_apt32f102_ept.o), (12 bytes).
	Removing .text.EPT_EPX_Config(Obj/FWlib_apt32f102_ept.o), (176 bytes).
	Removing .text.EPT_EPIX_POL_Config(Obj/FWlib_apt32f102_ept.o), (24 bytes).
	Removing .text.EPT_LKCR_TRG_Config(Obj/FWlib_apt32f102_ept.o), (120 bytes).
	Removing .text.EPT_SHLOCK_OUTPUT_Config(Obj/FWlib_apt32f102_ept.o), (28 bytes).
	Removing .text.EPT_SLock_CLR(Obj/FWlib_apt32f102_ept.o), (20 bytes).
	Removing .text.EPT_HLock_CLR(Obj/FWlib_apt32f102_ept.o), (20 bytes).
	Removing .text.EPT_SW_Set_lock(Obj/FWlib_apt32f102_ept.o), (28 bytes).
	Removing .text(Obj/FWlib_apt32f102_rtc.o), (0 bytes).
	Removing .data(Obj/FWlib_apt32f102_rtc.o), (0 bytes).
	Removing .bss(Obj/FWlib_apt32f102_rtc.o), (0 bytes).
	Removing .text.RTC_RST_VALUE(Obj/FWlib_apt32f102_rtc.o), (40 bytes).
	Removing .text.RTC_ALM_IO_SET(Obj/FWlib_apt32f102_rtc.o), (64 bytes).
	Removing .text.RTCCLK_CONFIG(Obj/FWlib_apt32f102_rtc.o), (72 bytes).
	Removing .text.RTC_Function_Config(Obj/FWlib_apt32f102_rtc.o), (44 bytes).
	Removing .text.RTC_Start(Obj/FWlib_apt32f102_rtc.o), (44 bytes).
	Removing .text.RTC_Stop(Obj/FWlib_apt32f102_rtc.o), (44 bytes).
	Removing .text.RTC_TIMR_DATR_SET(Obj/FWlib_apt32f102_rtc.o), (68 bytes).
	Removing .text.RTC_TIMR_DATR_Read(Obj/FWlib_apt32f102_rtc.o), (84 bytes).
	Removing .text.RTC_Alarm_TIMR_DATR_SET(Obj/FWlib_apt32f102_rtc.o), (172 bytes).
	Removing .text.RTC_AlarmA_TIMR_DATR_Read(Obj/FWlib_apt32f102_rtc.o), (60 bytes).
	Removing .text.RTC_AlarmB_TIMR_DATR_Read(Obj/FWlib_apt32f102_rtc.o), (60 bytes).
	Removing .text.RTC_TRGSRC0_Config(Obj/FWlib_apt32f102_rtc.o), (40 bytes).
	Removing .text.RTC_TRGSRC1_Config(Obj/FWlib_apt32f102_rtc.o), (40 bytes).
	Removing .text.RTC_TRGSRC0_SWFTRG(Obj/FWlib_apt32f102_rtc.o), (16 bytes).
	Removing .text.RTC_TRGSRC1_SWFTRG(Obj/FWlib_apt32f102_rtc.o), (16 bytes).
	Removing .text.RTC_Int_Enable(Obj/FWlib_apt32f102_rtc.o), (20 bytes).
	Removing .text.RTC_Int_Disable(Obj/FWlib_apt32f102_rtc.o), (16 bytes).
	Removing .text.RTC_Vector_Int_Enable(Obj/FWlib_apt32f102_rtc.o), (16 bytes).
	Removing .text.RTC_Vector_Int_Disable(Obj/FWlib_apt32f102_rtc.o), (16 bytes).
	Removing .text.RTC_WakeUp_Enable(Obj/FWlib_apt32f102_rtc.o), (16 bytes).
	Removing .text.RTC_WakeUp_Disable(Obj/FWlib_apt32f102_rtc.o), (16 bytes).
	Removing .debug_info(Obj/FWlib_apt32f102_rtc.o), (8815 bytes).
	Removing .debug_abbrev(Obj/FWlib_apt32f102_rtc.o), (494 bytes).
	Removing .debug_loc(Obj/FWlib_apt32f102_rtc.o), (535 bytes).
	Removing .debug_aranges(Obj/FWlib_apt32f102_rtc.o), (192 bytes).
	Removing .debug_ranges(Obj/FWlib_apt32f102_rtc.o), (176 bytes).
	Removing .debug_line(Obj/FWlib_apt32f102_rtc.o), (606 bytes).
	Removing .debug_str(Obj/FWlib_apt32f102_rtc.o), (4854 bytes).
	Removing .comment(Obj/FWlib_apt32f102_rtc.o), (67 bytes).
	Removing .debug_frame(Obj/FWlib_apt32f102_rtc.o), (428 bytes).
	Removing .csky.attributes(Obj/FWlib_apt32f102_rtc.o), (32 bytes).
	Removing COMMON(Obj/FWlib_apt32f102_rtc.o), (15 bytes).
	Removing .text(Obj/FWlib_apt32f102_adc.o), (0 bytes).
	Removing .data(Obj/FWlib_apt32f102_adc.o), (0 bytes).
	Removing .bss(Obj/FWlib_apt32f102_adc.o), (0 bytes).
	Removing .text.ADC12_RESET_VALUE(Obj/FWlib_apt32f102_adc.o), (100 bytes).
	Removing .text.ADC12_Control(Obj/FWlib_apt32f102_adc.o), (16 bytes).
	Removing .text.ADC12_CMD.part.0(Obj/FWlib_apt32f102_adc.o), (32 bytes).
	Removing .text.ADC12_ConfigInterrupt_CMD(Obj/FWlib_apt32f102_adc.o), (32 bytes).
	Removing .text.ADC12_Read_IntEnStatus(Obj/FWlib_apt32f102_adc.o), (20 bytes).
	Removing .text.ADC12_CLK_CMD(Obj/FWlib_apt32f102_adc.o), (44 bytes).
	Removing .text.ADC12_Software_Reset(Obj/FWlib_apt32f102_adc.o), (10 bytes).
	Removing .text.ADC12_CMD(Obj/FWlib_apt32f102_adc.o), (40 bytes).
	Removing .text.ADC12_ready_wait(Obj/FWlib_apt32f102_adc.o), (20 bytes).
	Removing .text.ADC12_EOC_wait(Obj/FWlib_apt32f102_adc.o), (20 bytes).
	Removing .text.ADC12_SEQEND_wait(Obj/FWlib_apt32f102_adc.o), (24 bytes).
	Removing .text.ADC12_DATA_OUPUT(Obj/FWlib_apt32f102_adc.o), (20 bytes).
	Removing .text.ADC12_Configure_Mode(Obj/FWlib_apt32f102_adc.o), (124 bytes).
	Removing .text.ADC12_Configure_VREF_Selecte(Obj/FWlib_apt32f102_adc.o), (408 bytes).
	Removing .text.ADC12_CompareFunction_set(Obj/FWlib_apt32f102_adc.o), (32 bytes).
	Removing .text.ADC12_ConversionChannel_Config(Obj/FWlib_apt32f102_adc.o), (384 bytes).
	Removing .text.ADC12_Compare_statue(Obj/FWlib_apt32f102_adc.o), (44 bytes).
	Removing .text.ADC_Int_Enable(Obj/FWlib_apt32f102_adc.o), (28 bytes).
	Removing .text.ADC_Int_Disable(Obj/FWlib_apt32f102_adc.o), (12 bytes).
	Removing .debug_info(Obj/FWlib_apt32f102_adc.o), (8666 bytes).
	Removing .debug_abbrev(Obj/FWlib_apt32f102_adc.o), (663 bytes).
	Removing .debug_loc(Obj/FWlib_apt32f102_adc.o), (936 bytes).
	Removing .debug_aranges(Obj/FWlib_apt32f102_adc.o), (176 bytes).
	Removing .debug_ranges(Obj/FWlib_apt32f102_adc.o), (160 bytes).
	Removing .debug_line(Obj/FWlib_apt32f102_adc.o), (684 bytes).
	Removing .debug_str(Obj/FWlib_apt32f102_adc.o), (4962 bytes).
	Removing .comment(Obj/FWlib_apt32f102_adc.o), (67 bytes).
	Removing .debug_frame(Obj/FWlib_apt32f102_adc.o), (400 bytes).
	Removing .csky.attributes(Obj/FWlib_apt32f102_adc.o), (32 bytes).
	Removing .text(Obj/FWlib_apt32f102_ifc.o), (0 bytes).
	Removing .data(Obj/FWlib_apt32f102_ifc.o), (0 bytes).
	Removing .bss(Obj/FWlib_apt32f102_ifc.o), (1 bytes).
	Removing .text.ChipErase(Obj/FWlib_apt32f102_ifc.o), (36 bytes).
	Removing .text.PageErase(Obj/FWlib_apt32f102_ifc.o), (36 bytes).
	Removing .text.Page_ProgramData_int(Obj/FWlib_apt32f102_ifc.o), (156 bytes).
	Removing .text.Page_ProgramData(Obj/FWlib_apt32f102_ifc.o), (160 bytes).
	Removing .text.Page_ProgramData_U32(Obj/FWlib_apt32f102_ifc.o), (124 bytes).
	Removing .text.ReadDataArry(Obj/FWlib_apt32f102_ifc.o), (46 bytes).
	Removing .text.ReadDataArry_U8(Obj/FWlib_apt32f102_ifc.o), (42 bytes).
	Removing .text.ReadDataArry_U32(Obj/FWlib_apt32f102_ifc.o), (22 bytes).
	Removing .text.IFC_interrupt_CMD(Obj/FWlib_apt32f102_ifc.o), (28 bytes).
	Removing .text.IFC_Int_Enable(Obj/FWlib_apt32f102_ifc.o), (28 bytes).
	Removing .text.IFC_Int_Disable(Obj/FWlib_apt32f102_ifc.o), (12 bytes).
	Removing .debug_info(Obj/FWlib_apt32f102_ifc.o), (9889 bytes).
	Removing .debug_abbrev(Obj/FWlib_apt32f102_ifc.o), (525 bytes).
	Removing .debug_loc(Obj/FWlib_apt32f102_ifc.o), (403 bytes).
	Removing .debug_aranges(Obj/FWlib_apt32f102_ifc.o), (112 bytes).
	Removing .debug_ranges(Obj/FWlib_apt32f102_ifc.o), (96 bytes).
	Removing .debug_line(Obj/FWlib_apt32f102_ifc.o), (470 bytes).
	Removing .debug_str(Obj/FWlib_apt32f102_ifc.o), (7611 bytes).
	Removing .comment(Obj/FWlib_apt32f102_ifc.o), (67 bytes).
	Removing .debug_frame(Obj/FWlib_apt32f102_ifc.o), (268 bytes).
	Removing .csky.attributes(Obj/FWlib_apt32f102_ifc.o), (32 bytes).
	Removing COMMON(Obj/FWlib_apt32f102_ifc.o), (4 bytes).
	Removing .text(Obj/FWlib_apt32f102_coret.o), (0 bytes).
	Removing .data(Obj/FWlib_apt32f102_coret.o), (0 bytes).
	Removing .bss(Obj/FWlib_apt32f102_coret.o), (0 bytes).
	Removing .text.CORET_DeInit(Obj/FWlib_apt32f102_coret.o), (24 bytes).
	Removing .text.CORET_Int_Enable(Obj/FWlib_apt32f102_coret.o), (24 bytes).
	Removing .text.CORET_Int_Disable(Obj/FWlib_apt32f102_coret.o), (12 bytes).
	Removing .text.CORET_WakeUp_Enable(Obj/FWlib_apt32f102_coret.o), (12 bytes).
	Removing .text.CORET_WakeUp_Disable(Obj/FWlib_apt32f102_coret.o), (12 bytes).
	Removing .text.CORET_start(Obj/FWlib_apt32f102_coret.o), (16 bytes).
	Removing .text.CORET_stop(Obj/FWlib_apt32f102_coret.o), (16 bytes).
	Removing .text.CORET_CLKSOURCE_EX(Obj/FWlib_apt32f102_coret.o), (16 bytes).
	Removing .text.CORET_CLKSOURCE_IN(Obj/FWlib_apt32f102_coret.o), (16 bytes).
	Removing .text.CORET_TICKINT_Enable(Obj/FWlib_apt32f102_coret.o), (16 bytes).
	Removing .text.CORET_TICKINT_Disable(Obj/FWlib_apt32f102_coret.o), (16 bytes).
	Removing .text.CORET_reload(Obj/FWlib_apt32f102_coret.o), (16 bytes).
	Removing .debug_info(Obj/FWlib_apt32f102_coret.o), (7132 bytes).
	Removing .debug_abbrev(Obj/FWlib_apt32f102_coret.o), (295 bytes).
	Removing .debug_aranges(Obj/FWlib_apt32f102_coret.o), (120 bytes).
	Removing .debug_ranges(Obj/FWlib_apt32f102_coret.o), (104 bytes).
	Removing .debug_line(Obj/FWlib_apt32f102_coret.o), (323 bytes).
	Removing .debug_str(Obj/FWlib_apt32f102_coret.o), (2860 bytes).
	Removing .comment(Obj/FWlib_apt32f102_coret.o), (67 bytes).
	Removing .debug_frame(Obj/FWlib_apt32f102_coret.o), (208 bytes).
	Removing .csky.attributes(Obj/FWlib_apt32f102_coret.o), (32 bytes).
	Removing .text(Obj/main.o), (0 bytes).
	Removing .data(Obj/main.o), (0 bytes).
	Removing .bss(Obj/main.o), (7 bytes).
	Removing .text(Obj/mcu_initial.o), (0 bytes).
	Removing .data(Obj/mcu_initial.o), (0 bytes).
	Removing .bss(Obj/mcu_initial.o), (0 bytes).
	Removing .text.GPIO_CONFIG(Obj/mcu_initial.o), (2 bytes).
	Removing .text.EPT0_CONFIG(Obj/mcu_initial.o), (108 bytes).
	Removing .text.GPT0_CONFIG(Obj/mcu_initial.o), (2 bytes).
	Removing .text.UART0_CONFIG(Obj/mcu_initial.o), (52 bytes).
	Removing .text.UART1_CONFIG(Obj/mcu_initial.o), (52 bytes).
	Removing .text.UART2_CONFIG(Obj/mcu_initial.o), (36 bytes).
	Removing .text.ADC12_CONFIG(Obj/mcu_initial.o), (114 bytes).
	Removing .text.SIO_CONFIG(Obj/mcu_initial.o), (64 bytes).
	Removing .text(Obj/mcu_interrupt.o), (0 bytes).
	Removing .data(Obj/mcu_interrupt.o), (1 bytes).
	Removing .text.SystemDesPtr(Obj/mcu_interrupt.o), (2 bytes).
	Removing .text(Obj/drivers_apt32f102.o), (0 bytes).
	Removing .bss(Obj/drivers_apt32f102.o), (0 bytes).
	Removing .text.__modsi3(Obj/drivers_apt32f102.o), (36 bytes).
	Removing .text(Obj/drivers_apt32f102_ck801.o), (0 bytes).
	Removing .data(Obj/drivers_apt32f102_ck801.o), (0 bytes).
	Removing .bss(Obj/drivers_apt32f102_ck801.o), (0 bytes).
	Removing .text.CK801_Init(Obj/drivers_apt32f102_ck801.o), (108 bytes).
	Removing .text.force_interrupt(Obj/drivers_apt32f102_ck801.o), (24 bytes).
	Removing .text(Obj/SYSTEM_uart.o), (0 bytes).
	Removing .data(Obj/SYSTEM_uart.o), (4 bytes).
	Removing .text.UART0_TASK(Obj/SYSTEM_uart.o), (60 bytes).
	Removing .text.UART2_RecvINT_Processing(Obj/SYSTEM_uart.o), (52 bytes).
	Removing .text.UART0_RecvINT_Processing(Obj/SYSTEM_uart.o), (8 bytes).
	Removing .text.UART2_TASK(Obj/SYSTEM_uart.o), (96 bytes).
	Removing .text.UART_Waiting_For_Send(Obj/SYSTEM_uart.o), (32 bytes).
	Removing .text.MCU485_SendData(Obj/SYSTEM_uart.o), (144 bytes).
	Removing .text.Clear_SendFlag(Obj/SYSTEM_uart.o), (16 bytes).
	Removing .text.BUS485_Jump_Boot(Obj/SYSTEM_uart.o), (12 bytes).
	Removing .text.Get_BUS485_Send_State(Obj/SYSTEM_uart.o), (28 bytes).
	Removing .text.Dbg_Print(Obj/SYSTEM_uart.o), (12 bytes).
	Removing .text.Dbg_Print_Buff(Obj/SYSTEM_uart.o), (2 bytes).
	Removing .text(Obj/SYSTEM_dip_switch.o), (0 bytes).
	Removing .data(Obj/SYSTEM_dip_switch.o), (0 bytes).
	Removing .text(Obj/SYSTEM_control_rly.o), (0 bytes).
	Removing .data(Obj/SYSTEM_control_rly.o), (0 bytes).
	Removing .bss(Obj/SYSTEM_control_rly.o), (0 bytes).
	Removing .text.CheckSum2(Obj/SYSTEM_control_rly.o), (24 bytes).
	Removing .text.BLV_WINDOUT_CMD_SET_Processing(Obj/SYSTEM_control_rly.o), (160 bytes).
	Removing .text.set_vol(Obj/SYSTEM_control_rly.o), (124 bytes).
	Removing .text(Obj/SYSTEM_eeprom.o), (0 bytes).
	Removing .data(Obj/SYSTEM_eeprom.o), (0 bytes).
	Removing .bss(Obj/SYSTEM_eeprom.o), (0 bytes).
	Removing .text.EEPROM_CheckSum(Obj/SYSTEM_eeprom.o), (22 bytes).
	Removing .text.EEPROM_ReadPara(Obj/SYSTEM_eeprom.o), (428 bytes).
	Removing .text.EEPROM_ValidateWrite(Obj/SYSTEM_eeprom.o), (116 bytes).
	Removing .text.EEPROM_WritePara(Obj/SYSTEM_eeprom.o), (164 bytes).
	Removing .text.EEPROM_ReadMCUDevInfo(Obj/SYSTEM_eeprom.o), (112 bytes).
	Removing .text.EEPROM_WriteMCUDevInfo(Obj/SYSTEM_eeprom.o), (64 bytes).
	Removing .text.EEPROM_Default_MCUDevInfo(Obj/SYSTEM_eeprom.o), (52 bytes).
	Removing .text.EEPROM_Validate_MCUDevInfo(Obj/SYSTEM_eeprom.o), (88 bytes).
	Removing .text.EEPROM_Init(Obj/SYSTEM_eeprom.o), (64 bytes).
	Removing .rodata.str1.1(Obj/SYSTEM_eeprom.o), (337 bytes).
	Removing .debug_info(Obj/SYSTEM_eeprom.o), (9839 bytes).
	Removing .debug_abbrev(Obj/SYSTEM_eeprom.o), (626 bytes).
	Removing .debug_loc(Obj/SYSTEM_eeprom.o), (403 bytes).
	Removing .debug_aranges(Obj/SYSTEM_eeprom.o), (96 bytes).
	Removing .debug_ranges(Obj/SYSTEM_eeprom.o), (104 bytes).
	Removing .debug_line(Obj/SYSTEM_eeprom.o), (806 bytes).
	Removing .debug_str(Obj/SYSTEM_eeprom.o), (4683 bytes).
	Removing .comment(Obj/SYSTEM_eeprom.o), (67 bytes).
	Removing .debug_frame(Obj/SYSTEM_eeprom.o), (280 bytes).
	Removing .csky.attributes(Obj/SYSTEM_eeprom.o), (32 bytes).
	Removing COMMON(Obj/SYSTEM_eeprom.o), (37 bytes).
	Removing .text(Obj/__rt_entry.o), (240 bytes).
	Removing .data(Obj/__rt_entry.o), (0 bytes).
	Removing .bss(Obj/__rt_entry.o), (0 bytes).
	Removing .debug_line(Obj/__rt_entry.o), (131 bytes).
	Removing .debug_info(Obj/__rt_entry.o), (125 bytes).
	Removing .debug_abbrev(Obj/__rt_entry.o), (20 bytes).
	Removing .debug_aranges(Obj/__rt_entry.o), (32 bytes).
	Removing .csky.attributes(Obj/__rt_entry.o), (32 bytes).
	Removing .text(FWlib_apt32f102_tkey_c_1_17.o), (0 bytes).
	Removing .bss(FWlib_apt32f102_tkey_c_1_17.o), (0 bytes).
	Removing .text.TK_ConfigInterrupt_CMD.part.0(FWlib_apt32f102_tkey_c_1_17.o), (16 bytes).
	Removing .text.TK_DeInit(FWlib_apt32f102_tkey_c_1_17.o), (60 bytes).
	Removing .text.tk_clk_config(FWlib_apt32f102_tkey_c_1_17.o), (40 bytes).
	Removing .text.TK_con0_config(FWlib_apt32f102_tkey_c_1_17.o), (188 bytes).
	Removing .text.tk_scan_config(FWlib_apt32f102_tkey_c_1_17.o), (40 bytes).
	Removing .text.TK_ConfigInterrupt_CMD(FWlib_apt32f102_tkey_c_1_17.o), (32 bytes).
	Removing .text.TK_IO_Enable(FWlib_apt32f102_tkey_c_1_17.o), (308 bytes).
	Removing .text.lpt_init(FWlib_apt32f102_tkey_c_1_17.o), (76 bytes).
	Removing .text.TK_setup_sleep(FWlib_apt32f102_tkey_c_1_17.o), (92 bytes).
	Removing .text.TK_quit_sleep(FWlib_apt32f102_tkey_c_1_17.o), (40 bytes).
	Removing .text.TK_Baseline_prog(FWlib_apt32f102_tkey_c_1_17.o), (132 bytes).
	Removing .text.get_key_seq(FWlib_apt32f102_tkey_c_1_17.o), (52 bytes).
	Removing .text.CORET_CONFIG(FWlib_apt32f102_tkey_c_1_17.o), (56 bytes).
	Removing .text.tk_chxval_seqxcon_clr(FWlib_apt32f102_tkey_c_1_17.o), (28 bytes).
	Removing .text.tk_reserved_init(FWlib_apt32f102_tkey_c_1_17.o), (40 bytes).
	Removing .text.tk_init(FWlib_apt32f102_tkey_c_1_17.o), (384 bytes).
	Removing .text(FWlib_apt32f102_clkcalib.o), (0 bytes).
	Removing .data(FWlib_apt32f102_clkcalib.o), (0 bytes).
	Removing .bss(FWlib_apt32f102_clkcalib.o), (0 bytes).
	Removing .data(pow.o), (0 bytes).
	Removing .bss(pow.o), (0 bytes).
	Removing .data(fabs.o), (0 bytes).
	Removing .bss(fabs.o), (0 bytes).
	Removing .data(scalbn.o), (0 bytes).
	Removing .bss(scalbn.o), (0 bytes).
	Removing .data(sqrt.o), (0 bytes).
	Removing .bss(sqrt.o), (0 bytes).
	Removing .data(_csky_case_uqi.o), (0 bytes).
	Removing .bss(_csky_case_uqi.o), (0 bytes).
	Removing .data(_fixunsdfsi.o), (0 bytes).
	Removing .bss(_fixunsdfsi.o), (0 bytes).
	Removing .data(_addsub_df.o), (0 bytes).
	Removing .bss(_addsub_df.o), (0 bytes).
	Removing .data(_mul_df.o), (0 bytes).
	Removing .bss(_mul_df.o), (0 bytes).
	Removing .data(_div_df.o), (0 bytes).
	Removing .bss(_div_df.o), (0 bytes).
	Removing .data(_gt_df.o), (0 bytes).
	Removing .bss(_gt_df.o), (0 bytes).
	Removing .data(_ge_df.o), (0 bytes).
	Removing .bss(_ge_df.o), (0 bytes).
	Removing .data(_le_df.o), (0 bytes).
	Removing .bss(_le_df.o), (0 bytes).
	Removing .data(_si_to_df.o), (0 bytes).
	Removing .bss(_si_to_df.o), (0 bytes).
	Removing .data(_df_to_si.o), (0 bytes).
	Removing .bss(_df_to_si.o), (0 bytes).
	Removing .text(_thenan_df.o), (0 bytes).
	Removing .data(_thenan_df.o), (0 bytes).
	Removing .bss(_thenan_df.o), (0 bytes).
	Removing .data(_usi_to_df.o), (0 bytes).
	Removing .bss(_usi_to_df.o), (0 bytes).
	Removing .data(_muldi3.o), (0 bytes).
	Removing .bss(_muldi3.o), (0 bytes).
	Removing .data(_clzsi2.o), (0 bytes).
	Removing .bss(_clzsi2.o), (0 bytes).
	Removing .data(_pack_df.o), (0 bytes).
	Removing .bss(_pack_df.o), (0 bytes).
	Removing .data(_unpack_df.o), (0 bytes).
	Removing .bss(_unpack_df.o), (0 bytes).
	Removing .data(_fpcmp_parts_df.o), (0 bytes).
	Removing .bss(_fpcmp_parts_df.o), (0 bytes).
	Removing .text(_clz.o), (0 bytes).
	Removing .data(_clz.o), (0 bytes).
	Removing .bss(_clz.o), (0 bytes).
	Removing .data(memset_fast.o), (0 bytes).
	Removing .bss(memset_fast.o), (0 bytes).
	Removing .data(memcpy_fast.o), (0 bytes).
	Removing .bss(memcpy_fast.o), (0 bytes).
	Removing .text(strncmp.o), (38 bytes).
	Removing .data(strncmp.o), (0 bytes).
	Removing .bss(strncmp.o), (0 bytes).
	Removing .csky.attributes(strncmp.o), (32 bytes).

633 unused seciton(s) (total 197032 bytes) removed from the image.

======================================================================

Image Symbol Table 

	Local Symbols

	Symbol Name                        Value        Type   Size  Section
	FWlib_apt32f102_clkcalib.o         0x00000000     df        0  *ABS*
	FWlib_apt32f102_tkey_c_1_17.o      0x00000000     df        0  *ABS*
	Obj/FWlib_apt32f102_bt.o           0x00000000     df        0  *ABS*
	Obj/FWlib_apt32f102_ept.o          0x00000000     df        0  *ABS*
	Obj/FWlib_apt32f102_gpio.o         0x00000000     df        0  *ABS*
	Obj/FWlib_apt32f102_gpt.o          0x00000000     df        0  *ABS*
	Obj/FWlib_apt32f102_lpt.o          0x00000000     df        0  *ABS*
	Obj/FWlib_apt32f102_syscon.o       0x00000000     df        0  *ABS*
	Obj/FWlib_apt32f102_uart.o         0x00000000     df        0  *ABS*
	Obj/FWlib_apt32f102_wwdt.o         0x00000000     df        0  *ABS*
	Obj/SYSTEM_control_rly.o           0x00000000     df        0  *ABS*
	Obj/SYSTEM_dip_switch.o            0x00000000     df        0  *ABS*
	Obj/SYSTEM_uart.o                  0x00000000     df        0  *ABS*
	Obj/arch_crt0.o                    0x00000000     df        0  *ABS*
	Obj/arch_mem_init.o                0x00000000     df        0  *ABS*
	Obj/drivers_apt32f102.o            0x00000000     df        0  *ABS*
	Obj/drivers_apt32f102_ck801.o      0x00000000     df        0  *ABS*
	Obj/main.o                         0x00000000     df        0  *ABS*
	Obj/mcu_initial.o                  0x00000000     df        0  *ABS*
	Obj/mcu_interrupt.o                0x00000000     df        0  *ABS*
	_addsub_df.o                       0x00000000     df        0  *ABS*
	_clzsi2.o                          0x00000000     df        0  *ABS*
	_csky_case_uqi.o                   0x00000000     df        0  *ABS*
	_df_to_si.o                        0x00000000     df        0  *ABS*
	_div_df.o                          0x00000000     df        0  *ABS*
	_fixunsdfsi.o                      0x00000000     df        0  *ABS*
	_fpcmp_parts_df.o                  0x00000000     df        0  *ABS*
	_ge_df.o                           0x00000000     df        0  *ABS*
	_gt_df.o                           0x00000000     df        0  *ABS*
	_le_df.o                           0x00000000     df        0  *ABS*
	_mul_df.o                          0x00000000     df        0  *ABS*
	_muldi3.o                          0x00000000     df        0  *ABS*
	_pack_df.o                         0x00000000     df        0  *ABS*
	_si_to_df.o                        0x00000000     df        0  *ABS*
	_unpack_df.o                       0x00000000     df        0  *ABS*
	_usi_to_df.o                       0x00000000     df        0  *ABS*
	fabs.o                             0x00000000     df        0  *ABS*
	memcpy_fast.o                      0x00000000     df        0  *ABS*
	memset_fast.o                      0x00000000     df        0  *ABS*
	pow.o                              0x00000000     df        0  *ABS*
	scalbn.o                           0x00000000     df        0  *ABS*
	sqrt.o                             0x00000000     df        0  *ABS*
	$d                                 0x00000000               0  .text
	$t                                 0x0000010c               0  .text
	INIT_KERLE_STACK                   0x0000013e               0  .text
	__to_main                          0x00000146               0  .text
	__dummy                            0x00000182               0  .text
	$d                                 0x00000186               0  .text
	$d                                 0x000001b4               0  .text
	$t                                 0x000001b4               0  .text
	$d                                 0x00000578               0  .text
	$t                                 0x000005e0               0  .text
	$d                                 0x00000aa8               0  .text
	$t                                 0x00000b58               0  .text
	$d                                 0x00000b5e               0  .text
	$t                                 0x00000b5e               0  .text
	$d                                 0x00000b64               0  .text
	$t                                 0x00000b64               0  .text
	$d                                 0x00000b80               0  .text
	$d                                 0x00000b84               0  .text
	$t                                 0x00000b84               0  .text
	$d                                 0x00000cf0               0  .text
	$d                                 0x00000cfc               0  .text
	$t                                 0x00000cfc               0  .text
	$d                                 0x00000d10               0  .text
	$t                                 0x00000d10               0  .text
	$d                                 0x00000d44               0  .text
	_fpadd_parts                       0x00000d48      F      724  .text
	$d                                 0x00000d48               0  .text
	$t                                 0x00000d48               0  .text
	$d                                 0x00001010               0  .text
	$t                                 0x0000101c               0  .text
	$d                                 0x00001084               0  .text
	$t                                 0x00001084               0  .text
	$d                                 0x000012ac               0  .text
	$d                                 0x000012b8               0  .text
	$t                                 0x000012b8               0  .text
	$d                                 0x00001408               0  .text
	$d                                 0x0000140c               0  .text
	$t                                 0x0000140c               0  .text
	$d                                 0x00001448               0  .text
	$t                                 0x00001448               0  .text
	$d                                 0x00001484               0  .text
	$t                                 0x00001484               0  .text
	$d                                 0x000014c0               0  .text
	$t                                 0x000014c0               0  .text
	$d                                 0x0000152c               0  .text
	$d                                 0x00001530               0  .text
	$t                                 0x00001530               0  .text
	$d                                 0x0000159c               0  .text
	$d                                 0x000015a0               0  .text
	$t                                 0x000015a0               0  .text
	$d                                 0x000015f4               0  .text
	$t                                 0x000015f4               0  .text
	$d                                 0x00001638               0  .text
	$t                                 0x00001638               0  .text
	$d                                 0x0000166c               0  .text
	$d                                 0x00001678               0  .text
	$t                                 0x00001678               0  .text
	$d                                 0x00001800               0  .text
	$d                                 0x00001814               0  .text
	$t                                 0x00001814               0  .text
	$d                                 0x000018cc               0  .text
	$d                                 0x000018d8               0  .text
	$t                                 0x000018d8               0  .text
	$d                                 0x00001964               0  .text
	$t                                 0x00001964               0  .text
	$d                                 0x000019ec               0  .text
	$t                                 0x000019ec               0  .text
	$d                                 0x00001a50               0  .text.__main
	$t                                 0x00001a50               0  .text.__main
	$d                                 0x00001a74               0  .text.__main
	SYSCON_General_CMD.part.0          0x00001a88      F      116  .text.SYSCON_General_CMD.part.0
	$d                                 0x00001a88               0  .text.SYSCON_General_CMD.part.0
	$t                                 0x00001a88               0  .text.SYSCON_General_CMD.part.0
	$d                                 0x00001af4               0  .text.SYSCON_General_CMD.part.0
	$d                                 0x00001afc               0  .text.SYSCON_RST_VALUE
	$t                                 0x00001afc               0  .text.SYSCON_RST_VALUE
	$d                                 0x00001b2c               0  .text.SYSCON_RST_VALUE
	$d                                 0x00001b48               0  .text.SYSCON_General_CMD
	$t                                 0x00001b48               0  .text.SYSCON_General_CMD
	$d                                 0x00001b74               0  .text.SYSCON_General_CMD
	$d                                 0x00001b78               0  .text.SystemCLK_HCLKDIV_PCLKDIV_Config
	$t                                 0x00001b78               0  .text.SystemCLK_HCLKDIV_PCLKDIV_Config
	$d                                 0x00001bf0               0  .text.SystemCLK_HCLKDIV_PCLKDIV_Config
	$d                                 0x00001c00               0  .text.SYSCON_HFOSC_SELECTE
	$t                                 0x00001c00               0  .text.SYSCON_HFOSC_SELECTE
	$d                                 0x00001c24               0  .text.SYSCON_HFOSC_SELECTE
	$d                                 0x00001c28               0  .text.SYSCON_WDT_CMD
	$t                                 0x00001c28               0  .text.SYSCON_WDT_CMD
	$d                                 0x00001c58               0  .text.SYSCON_WDT_CMD
	$d                                 0x00001c64               0  .text.SYSCON_IWDCNT_Reload
	$t                                 0x00001c64               0  .text.SYSCON_IWDCNT_Reload
	$d                                 0x00001c74               0  .text.SYSCON_IWDCNT_Reload
	$d                                 0x00001c78               0  .text.SYSCON_IWDCNT_Config
	$t                                 0x00001c78               0  .text.SYSCON_IWDCNT_Config
	$d                                 0x00001c88               0  .text.SYSCON_IWDCNT_Config
	$d                                 0x00001c90               0  .text.SYSCON_LVD_Config
	$t                                 0x00001c90               0  .text.SYSCON_LVD_Config
	$d                                 0x00001ca8               0  .text.SYSCON_LVD_Config
	$d                                 0x00001cb0               0  .text.LVD_Int_Enable
	$t                                 0x00001cb0               0  .text.LVD_Int_Enable
	$d                                 0x00001cc8               0  .text.LVD_Int_Enable
	$d                                 0x00001ccc               0  .text.IWDT_Int_Enable
	$t                                 0x00001ccc               0  .text.IWDT_Int_Enable
	$d                                 0x00001ce4               0  .text.IWDT_Int_Enable
	$d                                 0x00001ce8               0  .text.EXTI_trigger_CMD
	$t                                 0x00001ce8               0  .text.EXTI_trigger_CMD
	$d                                 0x00001d24               0  .text.EXTI_trigger_CMD
	$d                                 0x00001d28               0  .text.EXTI_interrupt_CMD
	$t                                 0x00001d28               0  .text.EXTI_interrupt_CMD
	$d                                 0x00001d54               0  .text.EXTI_interrupt_CMD
	$d                                 0x00001d5c               0  .text.GPIO_EXTI_interrupt
	$t                                 0x00001d5c               0  .text.GPIO_EXTI_interrupt
	$d                                 0x00001d60               0  .text.EXI4_Int_Enable
	$t                                 0x00001d60               0  .text.EXI4_Int_Enable
	$d                                 0x00001d6c               0  .text.EXI4_Int_Enable
	$d                                 0x00001d70               0  .text.SYSCON_Int_Enable
	$t                                 0x00001d70               0  .text.SYSCON_Int_Enable
	$d                                 0x00001d78               0  .text.SYSCON_Int_Enable
	$d                                 0x00001d7c               0  .text.SYSCON_Int_Disable
	$t                                 0x00001d7c               0  .text.SYSCON_Int_Disable
	$d                                 0x00001d84               0  .text.SYSCON_Int_Disable
	$d                                 0x00001d88               0  .text.SYSCON_INT_Priority
	$t                                 0x00001d88               0  .text.SYSCON_INT_Priority
	$d                                 0x00001da0               0  .text.SYSCON_INT_Priority
	$d                                 0x00001dac               0  .text.Set_INT_Priority
	$t                                 0x00001dac               0  .text.Set_INT_Priority
	$d                                 0x00001dd8               0  .text.Set_INT_Priority
	$d                                 0x00001ddc               0  .text.GPIO_Init
	$t                                 0x00001ddc               0  .text.GPIO_Init
	$d                                 0x00001dee               0  .text.GPIO_Init
	$t                                 0x00001df6               0  .text.GPIO_Init
	$d                                 0x00001e52               0  .text.GPIO_Init
	$t                                 0x00001e5a               0  .text.GPIO_Init
	$d                                 0x00001ea8               0  .text.GPIO_Init
	$d                                 0x00001ebc               0  .text.GPIO_PullHigh_Init
	$t                                 0x00001ebc               0  .text.GPIO_PullHigh_Init
	$d                                 0x00001ed0               0  .text.GPIO_DriveStrength_EN
	$t                                 0x00001ed0               0  .text.GPIO_DriveStrength_EN
	$d                                 0x00001ee0               0  .text.GPIO_IntGroup_Set
	$t                                 0x00001ee0               0  .text.GPIO_IntGroup_Set
	$d                                 0x00001fd4               0  .text.GPIO_IntGroup_Set
	$d                                 0x00001fec               0  .text.GPIOA0_EXI_Init
	$t                                 0x00001fec               0  .text.GPIOA0_EXI_Init
	$d                                 0x00001ff8               0  .text.GPIOA0_EXI_Init
	$t                                 0x00002008               0  .text.GPIOA0_EXI_Init
	$d                                 0x000020e4               0  .text.GPIOA0_EXI_Init
	$d                                 0x000020e8               0  .text.GPIO_Write_High
	$t                                 0x000020e8               0  .text.GPIO_Write_High
	$d                                 0x000020f0               0  .text.GPIO_Write_Low
	$t                                 0x000020f0               0  .text.GPIO_Write_Low
	$d                                 0x000020f8               0  .text.GPIO_Reverse
	$t                                 0x000020f8               0  .text.GPIO_Reverse
	$d                                 0x0000210e               0  .text.GPIO_Read_Status
	$t                                 0x0000210e               0  .text.GPIO_Read_Status
	$d                                 0x00002120               0  .text.LPT_Soft_Reset
	$t                                 0x00002120               0  .text.LPT_Soft_Reset
	$d                                 0x00002130               0  .text.LPT_Soft_Reset
	$d                                 0x00002134               0  .text.WWDT_CNT_Load
	$t                                 0x00002134               0  .text.WWDT_CNT_Load
	$d                                 0x00002140               0  .text.WWDT_CNT_Load
	$d                                 0x00002144               0  .text.BT_DeInit
	$t                                 0x00002144               0  .text.BT_DeInit
	$d                                 0x00002160               0  .text.BT_Start
	$t                                 0x00002160               0  .text.BT_Start
	$d                                 0x00002168               0  .text.BT_Soft_Reset
	$t                                 0x00002168               0  .text.BT_Soft_Reset
	$d                                 0x00002172               0  .text.BT_Configure
	$t                                 0x00002172               0  .text.BT_Configure
	$d                                 0x0000218a               0  .text.BT_ControlSet_Configure
	$t                                 0x0000218a               0  .text.BT_ControlSet_Configure
	$d                                 0x000021b6               0  .text.BT_Period_CMP_Write
	$t                                 0x000021b6               0  .text.BT_Period_CMP_Write
	$d                                 0x000021bc               0  .text.BT_ConfigInterrupt_CMD
	$t                                 0x000021bc               0  .text.BT_ConfigInterrupt_CMD
	$d                                 0x000021d0               0  .text.BT1_INT_ENABLE
	$t                                 0x000021d0               0  .text.BT1_INT_ENABLE
	$d                                 0x000021dc               0  .text.BT1_INT_ENABLE
	$d                                 0x000021e0               0  .text.GPT_IO_Init
	$t                                 0x000021e0               0  .text.GPT_IO_Init
	$d                                 0x00002278               0  .text.GPT_IO_Init
	$d                                 0x00002280               0  .text.GPT_Configure
	$t                                 0x00002280               0  .text.GPT_Configure
	$d                                 0x00002290               0  .text.GPT_Configure
	$d                                 0x00002294               0  .text.GPT_WaveCtrl_Configure
	$t                                 0x00002294               0  .text.GPT_WaveCtrl_Configure
	$d                                 0x000022d4               0  .text.GPT_WaveCtrl_Configure
	$d                                 0x000022d8               0  .text.GPT_WaveLoad_Configure
	$t                                 0x000022d8               0  .text.GPT_WaveLoad_Configure
	$d                                 0x000022e8               0  .text.GPT_WaveLoad_Configure
	$d                                 0x000022ec               0  .text.GPT_WaveOut_Configure
	$t                                 0x000022ec               0  .text.GPT_WaveOut_Configure
	$d                                 0x0000239c               0  .text.GPT_WaveOut_Configure
	$d                                 0x000023a0               0  .text.GPT_Start
	$t                                 0x000023a0               0  .text.GPT_Start
	$d                                 0x000023ac               0  .text.GPT_Start
	$d                                 0x000023b0               0  .text.GPT_Period_CMP_Write
	$t                                 0x000023b0               0  .text.GPT_Period_CMP_Write
	$d                                 0x000023bc               0  .text.GPT_Period_CMP_Write
	$d                                 0x000023c0               0  .text.GPT_ConfigInterrupt_CMD
	$t                                 0x000023c0               0  .text.GPT_ConfigInterrupt_CMD
	$d                                 0x000023d8               0  .text.GPT_ConfigInterrupt_CMD
	$d                                 0x000023dc               0  .text.UART0_DeInit
	$t                                 0x000023dc               0  .text.UART0_DeInit
	$d                                 0x000023f0               0  .text.UART0_DeInit
	$d                                 0x000023f4               0  .text.UART1_DeInit
	$t                                 0x000023f4               0  .text.UART1_DeInit
	$d                                 0x00002408               0  .text.UART1_DeInit
	$d                                 0x0000240c               0  .text.UART2_DeInit
	$t                                 0x0000240c               0  .text.UART2_DeInit
	$d                                 0x00002420               0  .text.UART2_DeInit
	$d                                 0x00002424               0  .text.UART1_Int_Enable
	$t                                 0x00002424               0  .text.UART1_Int_Enable
	$d                                 0x00002438               0  .text.UART1_Int_Enable
	$d                                 0x00002440               0  .text.UART2_Int_Enable
	$t                                 0x00002440               0  .text.UART2_Int_Enable
	$d                                 0x00002454               0  .text.UART2_Int_Enable
	$d                                 0x0000245c               0  .text.UART_IO_Init
	$t                                 0x0000245c               0  .text.UART_IO_Init
	$d                                 0x00002540               0  .text.UART_IO_Init
	$d                                 0x00002548               0  .text.UARTInitRxTxIntEn
	$t                                 0x00002548               0  .text.UARTInitRxTxIntEn
	$d                                 0x00002554               0  .text.UARTInitRxTxIntEn
	$d                                 0x00002558               0  .text.UARTTransmit
	$t                                 0x00002558               0  .text.UARTTransmit
	$d                                 0x00002578               0  .text.EPT_Stop
	$t                                 0x00002578               0  .text.EPT_Stop
	$d                                 0x00002598               0  .text.EPT_Stop
	$d                                 0x000025a0               0  .text.startup.main
	$t                                 0x000025a0               0  .text.startup.main
	$d                                 0x000025c0               0  .text.startup.main
	$d                                 0x000025c4               0  .text.delay_nms
	$t                                 0x000025c4               0  .text.delay_nms
	$d                                 0x000025f0               0  .text.delay_nus
	$t                                 0x000025f0               0  .text.delay_nus
	$d                                 0x00002614               0  .text.BT_CONFIG
	$t                                 0x00002614               0  .text.BT_CONFIG
	$d                                 0x0000266c               0  .text.BT_CONFIG
	$d                                 0x00002674               0  .text.SYSCON_CONFIG
	$t                                 0x00002674               0  .text.SYSCON_CONFIG
	$d                                 0x000026d8               0  .text.APT32F102_init
	$t                                 0x000026d8               0  .text.APT32F102_init
	$d                                 0x00002718               0  .text.APT32F102_init
	$d                                 0x00002724               0  .text.SYSCONIntHandler
	$t                                 0x00002724               0  .text.SYSCONIntHandler
	$d                                 0x00002810               0  .text.SYSCONIntHandler
	$d                                 0x00002814               0  .text.IFCIntHandler
	$t                                 0x00002814               0  .text.IFCIntHandler
	$d                                 0x00002878               0  .text.IFCIntHandler
	$d                                 0x0000287c               0  .text.ADCIntHandler
	$t                                 0x0000287c               0  .text.ADCIntHandler
	$d                                 0x000028e0               0  .text.ADCIntHandler
	$d                                 0x000028e4               0  .text.EPT0IntHandler
	$t                                 0x000028e4               0  .text.EPT0IntHandler
	$d                                 0x00002a84               0  .text.EPT0IntHandler
	$d                                 0x00002a90               0  .text.WWDTHandler
	$t                                 0x00002a90               0  .text.WWDTHandler
	$d                                 0x00002ac0               0  .text.WWDTHandler
	$d                                 0x00002ac4               0  .text.GPT0IntHandler
	$t                                 0x00002ac4               0  .text.GPT0IntHandler
	$d                                 0x00002b40               0  .text.GPT0IntHandler
	$d                                 0x00002b44               0  .text.RTCIntHandler
	$t                                 0x00002b44               0  .text.RTCIntHandler
	$d                                 0x00002bac               0  .text.RTCIntHandler
	$d                                 0x00002bb4               0  .text.UART0IntHandler
	$t                                 0x00002bb4               0  .text.UART0IntHandler
	$d                                 0x00002bec               0  .text.UART0IntHandler
	$d                                 0x00002bf0               0  .text.UART1IntHandler
	$t                                 0x00002bf0               0  .text.UART1IntHandler
	$d                                 0x00002c70               0  .text.UART1IntHandler
	$d                                 0x00002c84               0  .text.UART2IntHandler
	$t                                 0x00002c84               0  .text.UART2IntHandler
	$d                                 0x00002ccc               0  .text.UART2IntHandler
	$d                                 0x00002cd0               0  .text.SPI0IntHandler
	$t                                 0x00002cd0               0  .text.SPI0IntHandler
	$d                                 0x00002db4               0  .text.SPI0IntHandler
	$d                                 0x00002db8               0  .text.SIO0IntHandler
	$t                                 0x00002db8               0  .text.SIO0IntHandler
	$d                                 0x00002e08               0  .text.SIO0IntHandler
	$d                                 0x00002e0c               0  .text.EXI0IntHandler
	$t                                 0x00002e0c               0  .text.EXI0IntHandler
	$d                                 0x00002e38               0  .text.EXI0IntHandler
	$d                                 0x00002e3c               0  .text.EXI1IntHandler
	$t                                 0x00002e3c               0  .text.EXI1IntHandler
	$d                                 0x00002e68               0  .text.EXI1IntHandler
	$d                                 0x00002e6c               0  .text.EXI2to3IntHandler
	$t                                 0x00002e6c               0  .text.EXI2to3IntHandler
	$d                                 0x00002eb0               0  .text.EXI2to3IntHandler
	$d                                 0x00002eb4               0  .text.EXI4to9IntHandler
	$t                                 0x00002eb4               0  .text.EXI4to9IntHandler
	$d                                 0x00002ed0               0  .text.EXI4to9IntHandler
	$d                                 0x00002ed4               0  .text.EXI10to15IntHandler
	$t                                 0x00002ed4               0  .text.EXI10to15IntHandler
	$d                                 0x00002f3c               0  .text.EXI10to15IntHandler
	$d                                 0x00002f40               0  .text.LPTIntHandler
	$t                                 0x00002f40               0  .text.LPTIntHandler
	$d                                 0x00002f70               0  .text.LPTIntHandler
	$d                                 0x00002f74               0  .text.BT0IntHandler
	$t                                 0x00002f74               0  .text.BT0IntHandler
	$d                                 0x00002fbc               0  .text.BT0IntHandler
	$d                                 0x00002fc0               0  .text.BT1IntHandler
	$t                                 0x00002fc0               0  .text.BT1IntHandler
	$d                                 0x00003028               0  .text.BT1IntHandler
	$d                                 0x00003030               0  .text.PriviledgeVioHandler
	$t                                 0x00003030               0  .text.PriviledgeVioHandler
	$d                                 0x00003032               0  .text.PendTrapHandler
	$t                                 0x00003032               0  .text.PendTrapHandler
	$d                                 0x0000303a               0  .text.Trap3Handler
	$t                                 0x0000303a               0  .text.Trap3Handler
	$d                                 0x00003042               0  .text.Trap2Handler
	$t                                 0x00003042               0  .text.Trap2Handler
	$d                                 0x0000304a               0  .text.Trap1Handler
	$t                                 0x0000304a               0  .text.Trap1Handler
	$d                                 0x00003052               0  .text.Trap0Handler
	$t                                 0x00003052               0  .text.Trap0Handler
	$d                                 0x0000305a               0  .text.UnrecExecpHandler
	$t                                 0x0000305a               0  .text.UnrecExecpHandler
	$d                                 0x00003062               0  .text.BreakPointHandler
	$t                                 0x00003062               0  .text.BreakPointHandler
	$d                                 0x0000306a               0  .text.AccessErrHandler
	$t                                 0x0000306a               0  .text.AccessErrHandler
	$d                                 0x00003072               0  .text.IllegalInstrHandler
	$t                                 0x00003072               0  .text.IllegalInstrHandler
	$d                                 0x0000307a               0  .text.MisalignedHandler
	$t                                 0x0000307a               0  .text.MisalignedHandler
	$d                                 0x00003082               0  .text.CNTAIntHandler
	$t                                 0x00003082               0  .text.CNTAIntHandler
	$d                                 0x0000308a               0  .text.I2CIntHandler
	$t                                 0x0000308a               0  .text.I2CIntHandler
	$d                                 0x00003094               0  .text.__divsi3
	$t                                 0x00003094               0  .text.__divsi3
	$d                                 0x000030b4               0  .text.__divsi3
	$d                                 0x000030b8               0  .text.__udivsi3
	$t                                 0x000030b8               0  .text.__udivsi3
	$d                                 0x000030d8               0  .text.__udivsi3
	$d                                 0x000030dc               0  .text.__umodsi3
	$t                                 0x000030dc               0  .text.__umodsi3
	$d                                 0x000030fc               0  .text.__umodsi3
	$d                                 0x00003100               0  .text.CK_CPU_EnAllNormalIrq
	$t                                 0x00003100               0  .text.CK_CPU_EnAllNormalIrq
	$d                                 0x00003106               0  .text.CK_CPU_DisAllNormalIrq
	$t                                 0x00003106               0  .text.CK_CPU_DisAllNormalIrq
	$d                                 0x0000310c               0  .text.UARTx_Init
	$t                                 0x0000310c               0  .text.UARTx_Init
	$d                                 0x00003204               0  .text.UARTx_Init
	$d                                 0x0000322c               0  .text.UART1_RecvINT_Processing
	$t                                 0x0000322c               0  .text.UART1_RecvINT_Processing
	$d                                 0x00003254               0  .text.UART1_RecvINT_Processing
	$d                                 0x00003260               0  .text.UART1_TASK
	$t                                 0x00003260               0  .text.UART1_TASK
	$d                                 0x000032b0               0  .text.UART1_TASK
	$d                                 0x000032c0               0  .text.BUS485_Send
	$t                                 0x000032c0               0  .text.BUS485_Send
	$d                                 0x00003370               0  .text.BUS485_Send
	$d                                 0x00003384               0  .text.MultSend_Task
	$t                                 0x00003384               0  .text.MultSend_Task
	$d                                 0x000033e0               0  .text.MultSend_Task
	$d                                 0x000033e8               0  .text.Set_GroupSend
	$t                                 0x000033e8               0  .text.Set_GroupSend
	$d                                 0x00003438               0  .text.Set_GroupSend
	$d                                 0x00003444               0  .text.BUS485Send_Task
	$t                                 0x00003444               0  .text.BUS485Send_Task
	$d                                 0x00003468               0  .text.BUS485Send_Task
	$d                                 0x00003470               0  .text.BusIdle_Task
	$t                                 0x00003470               0  .text.BusIdle_Task
	$d                                 0x000034a4               0  .text.BusIdle_Task
	$d                                 0x000034ac               0  .text.BusBusy_Task
	$t                                 0x000034ac               0  .text.BusBusy_Task
	$d                                 0x000034f4               0  .text.BusBusy_Task
	$d                                 0x00003500               0  .text.Dbg_Println
	$t                                 0x00003500               0  .text.Dbg_Println
	$d                                 0x0000350c               0  .text.DIP_GetSwitchState
	$t                                 0x0000350c               0  .text.DIP_GetSwitchState
	$d                                 0x0000353c               0  .text.DIP_GetSwitchState
	$d                                 0x00003540               0  .text.DIP_Switch_Init
	$t                                 0x00003540               0  .text.DIP_Switch_Init
	$d                                 0x000035c0               0  .text.DIP_Switch_Init
	$d                                 0x000035cc               0  .text.DIP_ScanTask
	$t                                 0x000035cc               0  .text.DIP_ScanTask
	$d                                 0x0000364c               0  .text.DIP_ScanTask
	$d                                 0x00003658               0  .text.Relay_Init
	$t                                 0x00003658               0  .text.Relay_Init
	$d                                 0x00003710               0  .text.Relay_Init
	$d                                 0x00003724               0  .text.CheckSum
	$t                                 0x00003724               0  .text.CheckSum
	$d                                 0x0000373c               0  .text.Change_OUTV
	$t                                 0x0000373c               0  .text.Change_OUTV
	$d                                 0x00003750               0  .text.Change_OUTV
	$d                                 0x00003758               0  .text.BLV_VolOut_Ctrl
	$t                                 0x00003758               0  .text.BLV_VolOut_Ctrl
	$d                                 0x000037d4               0  .text.BLV_VolOut_Ctrl
	$d                                 0x000037e8               0  .text.BLV_RLY_Ctrl_Purpose
	$t                                 0x000037e8               0  .text.BLV_RLY_Ctrl_Purpose
	$d                                 0x0000385c               0  .text.BLV_RLY_Ctrl_Purpose
	$d                                 0x00003864               0  .text.BLV_RLY_Task
	$t                                 0x00003864               0  .text.BLV_RLY_Task
	$d                                 0x000038b0               0  .text.BLV_RLY_Task
	$d                                 0x000038b8               0  .text.BLV_A9RLY_CMD_SET_Processing
	$t                                 0x000038b8               0  .text.BLV_A9RLY_CMD_SET_Processing
	$d                                 0x0000394c               0  .text.BLV_A9RLY_CMD_SET_Processing
	$d                                 0x00003954               0  .text.BLV_A9RLY_CMD_READ_Processing
	$t                                 0x00003954               0  .text.BLV_A9RLY_CMD_READ_Processing
	$d                                 0x000039c4               0  .text.BLV_A9RLY_CMD_READ_Processing
	$d                                 0x000039cc               0  .text.BLV_RLY_RS485_Pro
	$t                                 0x000039cc               0  .text.BLV_RLY_RS485_Pro
	$d                                 0x00003a64               0  .text.BLV_RLY_RS485_Pro
	$d                                 0x00003a7c               0  .text.TK_Sampling_prog
	$t                                 0x00003a7c               0  .text.TK_Sampling_prog
	$d                                 0x00003ac4               0  .text.TK_Sampling_prog
	$d                                 0x00003ad4               0  .text.TKEYIntHandler
	$t                                 0x00003ad4               0  .text.TKEYIntHandler
	$d                                 0x00003b50               0  .text.TKEYIntHandler
	$d                                 0x00003b5c               0  .text.get_key_number
	$t                                 0x00003b5c               0  .text.get_key_number
	$d                                 0x00003b80               0  .text.get_key_number
	$d                                 0x00003b84               0  .text.TK_Scan_Start
	$t                                 0x00003b84               0  .text.TK_Scan_Start
	$d                                 0x00003b9c               0  .text.TK_Scan_Start
	$d                                 0x00003ba4               0  .text.TK_Keymap_prog
	$t                                 0x00003ba4               0  .text.TK_Keymap_prog
	$d                                 0x00003cec               0  .text.TK_Keymap_prog
	$d                                 0x00003d24               0  .text.TK_overflow_predict
	$t                                 0x00003d24               0  .text.TK_overflow_predict
	$d                                 0x00003e0c               0  .text.TK_overflow_predict
	$d                                 0x00003e40               0  .text.TK_Baseline_tracking
	$t                                 0x00003e40               0  .text.TK_Baseline_tracking
	$d                                 0x00003fe4               0  .text.TK_Baseline_tracking
	$d                                 0x00004010               0  .text.TK_result_prog
	$t                                 0x00004010               0  .text.TK_result_prog
	$d                                 0x00004050               0  .text.TK_result_prog
	$d                                 0x00004064               0  .text.CORETHandler
	$t                                 0x00004064               0  .text.CORETHandler
	$d                                 0x000040c4               0  .text.CORETHandler
	$d                                 0x000040dc               0  .text.std_clk_calib
	$t                                 0x000040dc               0  .text.std_clk_calib
	$d                                 0x00004324               0  .text.std_clk_calib
	bp                                 0x00004360      O       16  .rodata
	dp_l                               0x00004370      O       16  .rodata
	dp_h                               0x00004380      O       16  .rodata
	NUM.6030                           0x2000009c      O        1  .bss
	update_20ms.5936                   0x200000b8      O        4  .bss

	Global Symbols

	Symbol Name                        Value        Type   Size  Section
	vector_table                       0x00000000               0  .text
	__start                            0x0000010c               0  .text
	__exit                             0x00000160               0  .text
	__fail                             0x00000176               0  .text
	DummyHandler                       0x00000184               0  .text
	__GI_pow                           0x000001b4      F     2474  .text
	pow                                0x000001b4      F     2474  .text
	__GI_fabs                          0x00000b5e      F        6  .text
	fabs                               0x00000b5e      F        6  .text
	__GI_scalbn                        0x00000b64      F       32  .text
	scalbn                             0x00000b64      F       32  .text
	__GI_sqrt                          0x00000b84      F      376  .text
	sqrt                               0x00000b84      F      376  .text
	___gnu_csky_case_uqi               0x00000cfc      F       20  .text
	__fixunsdfsi                       0x00000d10      F       56  .text
	__adddf3                           0x0000101c      F       46  .text
	__subdf3                           0x0000104c      F       54  .text
	__muldf3                           0x00001084      F      564  .text
	__divdf3                           0x000012b8      F      340  .text
	__gtdf2                            0x0000140c      F       60  .text
	__gedf2                            0x00001448      F       60  .text
	__ledf2                            0x00001484      F       58  .text
	__floatsidf                        0x000014c0      F      112  .text
	__fixdfsi                          0x00001530      F      112  .text
	__floatunsidf                      0x000015a0      F       84  .text
	__muldi3                           0x000015f4      F       68  .text
	__clzsi2                           0x00001638      F       64  .text
	__pack_d                           0x00001678      F      412  .text
	__unpack_d                         0x00001814      F      196  .text
	__fpcmp_parts_d                    0x000018d8      F      140  .text
	__memset_fast                      0x00001964    w F      136  .text
	memset                             0x00001964    w F      136  .text
	__memcpy_fast                      0x000019ec    w F      100  .text
	memcpy                             0x000019ec    w F      100  .text
	__main                             0x00001a50      F       56  .text.__main
	SYSCON_RST_VALUE                   0x00001afc      F       76  .text.SYSCON_RST_VALUE
	SYSCON_General_CMD                 0x00001b48      F       48  .text.SYSCON_General_CMD
	SystemCLK_HCLKDIV_PCLKDIV_Config   0x00001b78      F      136  .text.SystemCLK_HCLKDIV_PCLKDIV_Config
	SYSCON_HFOSC_SELECTE               0x00001c00      F       40  .text.SYSCON_HFOSC_SELECTE
	SYSCON_WDT_CMD                     0x00001c28      F       60  .text.SYSCON_WDT_CMD
	SYSCON_IWDCNT_Reload               0x00001c64      F       20  .text.SYSCON_IWDCNT_Reload
	SYSCON_IWDCNT_Config               0x00001c78      F       24  .text.SYSCON_IWDCNT_Config
	SYSCON_LVD_Config                  0x00001c90      F       32  .text.SYSCON_LVD_Config
	LVD_Int_Enable                     0x00001cb0      F       28  .text.LVD_Int_Enable
	IWDT_Int_Enable                    0x00001ccc      F       28  .text.IWDT_Int_Enable
	EXTI_trigger_CMD                   0x00001ce8      F       64  .text.EXTI_trigger_CMD
	EXTI_interrupt_CMD                 0x00001d28      F       52  .text.EXTI_interrupt_CMD
	GPIO_EXTI_interrupt                0x00001d5c      F        4  .text.GPIO_EXTI_interrupt
	EXI4_Int_Enable                    0x00001d60      F       16  .text.EXI4_Int_Enable
	SYSCON_Int_Enable                  0x00001d70      F       12  .text.SYSCON_Int_Enable
	SYSCON_Int_Disable                 0x00001d7c      F       12  .text.SYSCON_Int_Disable
	SYSCON_INT_Priority                0x00001d88      F       36  .text.SYSCON_INT_Priority
	Set_INT_Priority                   0x00001dac      F       48  .text.Set_INT_Priority
	GPIO_Init                          0x00001ddc      F      224  .text.GPIO_Init
	GPIO_PullHigh_Init                 0x00001ebc      F       20  .text.GPIO_PullHigh_Init
	GPIO_DriveStrength_EN              0x00001ed0      F       14  .text.GPIO_DriveStrength_EN
	GPIO_IntGroup_Set                  0x00001ee0      F      268  .text.GPIO_IntGroup_Set
	GPIOA0_EXI_Init                    0x00001fec      F      252  .text.GPIOA0_EXI_Init
	GPIO_Write_High                    0x000020e8      F        8  .text.GPIO_Write_High
	GPIO_Write_Low                     0x000020f0      F        8  .text.GPIO_Write_Low
	GPIO_Reverse                       0x000020f8      F       22  .text.GPIO_Reverse
	GPIO_Read_Status                   0x0000210e      F       16  .text.GPIO_Read_Status
	LPT_Soft_Reset                     0x00002120      F       20  .text.LPT_Soft_Reset
	WWDT_CNT_Load                      0x00002134      F       16  .text.WWDT_CNT_Load
	BT_DeInit                          0x00002144      F       28  .text.BT_DeInit
	BT_Start                           0x00002160      F        8  .text.BT_Start
	BT_Soft_Reset                      0x00002168      F       10  .text.BT_Soft_Reset
	BT_Configure                       0x00002172      F       24  .text.BT_Configure
	BT_ControlSet_Configure            0x0000218a      F       44  .text.BT_ControlSet_Configure
	BT_Period_CMP_Write                0x000021b6      F        6  .text.BT_Period_CMP_Write
	BT_ConfigInterrupt_CMD             0x000021bc      F       18  .text.BT_ConfigInterrupt_CMD
	BT1_INT_ENABLE                     0x000021d0      F       16  .text.BT1_INT_ENABLE
	GPT_IO_Init                        0x000021e0      F      160  .text.GPT_IO_Init
	GPT_Configure                      0x00002280      F       20  .text.GPT_Configure
	GPT_WaveCtrl_Configure             0x00002294      F       68  .text.GPT_WaveCtrl_Configure
	GPT_WaveLoad_Configure             0x000022d8      F       20  .text.GPT_WaveLoad_Configure
	GPT_WaveOut_Configure              0x000022ec      F      180  .text.GPT_WaveOut_Configure
	GPT_Start                          0x000023a0      F       16  .text.GPT_Start
	GPT_Period_CMP_Write               0x000023b0      F       16  .text.GPT_Period_CMP_Write
	GPT_ConfigInterrupt_CMD            0x000023c0      F       28  .text.GPT_ConfigInterrupt_CMD
	UART0_DeInit                       0x000023dc      F       24  .text.UART0_DeInit
	UART1_DeInit                       0x000023f4      F       24  .text.UART1_DeInit
	UART2_DeInit                       0x0000240c      F       24  .text.UART2_DeInit
	UART1_Int_Enable                   0x00002424      F       28  .text.UART1_Int_Enable
	UART2_Int_Enable                   0x00002440      F       28  .text.UART2_Int_Enable
	UART_IO_Init                       0x0000245c      F      236  .text.UART_IO_Init
	UARTInitRxTxIntEn                  0x00002548      F       16  .text.UARTInitRxTxIntEn
	UARTTransmit                       0x00002558      F       30  .text.UARTTransmit
	EPT_Stop                           0x00002578      F       40  .text.EPT_Stop
	main                               0x000025a0      F       36  .text.startup.main
	delay_nms                          0x000025c4      F       44  .text.delay_nms
	delay_nus                          0x000025f0      F       34  .text.delay_nus
	BT_CONFIG                          0x00002614      F       96  .text.BT_CONFIG
	SYSCON_CONFIG                      0x00002674      F       98  .text.SYSCON_CONFIG
	APT32F102_init                     0x000026d8      F       76  .text.APT32F102_init
	SYSCONIntHandler                   0x00002724      F      240  .text.SYSCONIntHandler
	IFCIntHandler                      0x00002814      F      104  .text.IFCIntHandler
	ADCIntHandler                      0x0000287c      F      104  .text.ADCIntHandler
	EPT0IntHandler                     0x000028e4      F      428  .text.EPT0IntHandler
	WWDTHandler                        0x00002a90      F       52  .text.WWDTHandler
	GPT0IntHandler                     0x00002ac4      F      128  .text.GPT0IntHandler
	RTCIntHandler                      0x00002b44      F      112  .text.RTCIntHandler
	UART0IntHandler                    0x00002bb4      F       60  .text.UART0IntHandler
	UART1IntHandler                    0x00002bf0      F      148  .text.UART1IntHandler
	UART2IntHandler                    0x00002c84      F       76  .text.UART2IntHandler
	SPI0IntHandler                     0x00002cd0      F      232  .text.SPI0IntHandler
	SIO0IntHandler                     0x00002db8      F       84  .text.SIO0IntHandler
	EXI0IntHandler                     0x00002e0c      F       48  .text.EXI0IntHandler
	EXI1IntHandler                     0x00002e3c      F       48  .text.EXI1IntHandler
	EXI2to3IntHandler                  0x00002e6c      F       72  .text.EXI2to3IntHandler
	EXI4to9IntHandler                  0x00002eb4      F       32  .text.EXI4to9IntHandler
	EXI10to15IntHandler                0x00002ed4      F      108  .text.EXI10to15IntHandler
	LPTIntHandler                      0x00002f40      F       52  .text.LPTIntHandler
	BT0IntHandler                      0x00002f74      F       76  .text.BT0IntHandler
	BT1IntHandler                      0x00002fc0      F      112  .text.BT1IntHandler
	PriviledgeVioHandler               0x00003030      F        2  .text.PriviledgeVioHandler
	PendTrapHandler                    0x00003032      F        8  .text.PendTrapHandler
	Trap3Handler                       0x0000303a      F        8  .text.Trap3Handler
	Trap2Handler                       0x00003042      F        8  .text.Trap2Handler
	Trap1Handler                       0x0000304a      F        8  .text.Trap1Handler
	Trap0Handler                       0x00003052      F        8  .text.Trap0Handler
	UnrecExecpHandler                  0x0000305a      F        8  .text.UnrecExecpHandler
	BreakPointHandler                  0x00003062      F        8  .text.BreakPointHandler
	AccessErrHandler                   0x0000306a      F        8  .text.AccessErrHandler
	IllegalInstrHandler                0x00003072      F        8  .text.IllegalInstrHandler
	MisalignedHandler                  0x0000307a      F        8  .text.MisalignedHandler
	CNTAIntHandler                     0x00003082      F        8  .text.CNTAIntHandler
	I2CIntHandler                      0x0000308a      F        8  .text.I2CIntHandler
	__divsi3                           0x00003094      F       36  .text.__divsi3
	__udivsi3                          0x000030b8      F       36  .text.__udivsi3
	__umodsi3                          0x000030dc      F       36  .text.__umodsi3
	CK_CPU_EnAllNormalIrq              0x00003100      F        6  .text.CK_CPU_EnAllNormalIrq
	CK_CPU_DisAllNormalIrq             0x00003106      F        6  .text.CK_CPU_DisAllNormalIrq
	UARTx_Init                         0x0000310c      F      288  .text.UARTx_Init
	UART1_RecvINT_Processing           0x0000322c      F       52  .text.UART1_RecvINT_Processing
	UART1_TASK                         0x00003260      F       96  .text.UART1_TASK
	BUS485_Send                        0x000032c0      F      196  .text.BUS485_Send
	MultSend_Task                      0x00003384      F      100  .text.MultSend_Task
	Set_GroupSend                      0x000033e8      F       92  .text.Set_GroupSend
	BUS485Send_Task                    0x00003444      F       44  .text.BUS485Send_Task
	BusIdle_Task                       0x00003470      F       60  .text.BusIdle_Task
	BusBusy_Task                       0x000034ac      F       84  .text.BusBusy_Task
	Dbg_Println                        0x00003500      F       12  .text.Dbg_Println
	DIP_GetSwitchState                 0x0000350c      F       52  .text.DIP_GetSwitchState
	DIP_Switch_Init                    0x00003540      F      140  .text.DIP_Switch_Init
	DIP_ScanTask                       0x000035cc      F      140  .text.DIP_ScanTask
	Relay_Init                         0x00003658      F      196  .text.Relay_Init
	CheckSum                           0x00003724      F       22  .text.CheckSum
	Change_OUTV                        0x0000373c      F       28  .text.Change_OUTV
	BLV_VolOut_Ctrl                    0x00003758      F      144  .text.BLV_VolOut_Ctrl
	BLV_RLY_Ctrl_Purpose               0x000037e8      F      124  .text.BLV_RLY_Ctrl_Purpose
	BLV_RLY_Task                       0x00003864      F       84  .text.BLV_RLY_Task
	BLV_A9RLY_CMD_SET_Processing       0x000038b8      F      156  .text.BLV_A9RLY_CMD_SET_Processing
	BLV_A9RLY_CMD_READ_Processing      0x00003954      F      120  .text.BLV_A9RLY_CMD_READ_Processing
	BLV_RLY_RS485_Pro                  0x000039cc      F      176  .text.BLV_RLY_RS485_Pro
	TK_Sampling_prog                   0x00003a7c      F       88  .text.TK_Sampling_prog
	TKEYIntHandler                     0x00003ad4      F      136  .text.TKEYIntHandler
	get_key_number                     0x00003b5c      F       40  .text.get_key_number
	TK_Scan_Start                      0x00003b84      F       32  .text.TK_Scan_Start
	TK_Keymap_prog                     0x00003ba4      F      384  .text.TK_Keymap_prog
	TK_overflow_predict                0x00003d24      F      284  .text.TK_overflow_predict
	TK_Baseline_tracking               0x00003e40      F      464  .text.TK_Baseline_tracking
	TK_result_prog                     0x00004010      F       84  .text.TK_result_prog
	CORETHandler                       0x00004064      F      120  .text.CORETHandler
	std_clk_calib                      0x000040dc      F      644  .text.std_clk_calib
	__thenan_df                        0x00004390      O       20  .rodata
	__clz_tab                          0x000043a4      O      256  .rodata
	_end_rodata                        0x00004560               0  .rodata
	HWD                                0x20000000      O        4  .data
	_start_data                        0x20000000               0  .data
	CRC                                0x20000004      O        4  .data
	BT1                                0x20000008      O        4  .data
	BT0                                0x2000000c      O        4  .data
	WWDT                               0x20000010      O        4  .data
	LPT                                0x20000014      O        4  .data
	RTC                                0x20000018      O        4  .data
	ETCB                               0x2000001c      O        4  .data
	EPT0                               0x20000020      O        4  .data
	GPT0                               0x20000024      O        4  .data
	CA0                                0x20000028      O        4  .data
	SIO0                               0x2000002c      O        4  .data
	I2C0                               0x20000030      O        4  .data
	SPI0                               0x20000034      O        4  .data
	UART2                              0x20000038      O        4  .data
	UART1                              0x2000003c      O        4  .data
	UART0                              0x20000040      O        4  .data
	GPIOGRP                            0x20000044      O        4  .data
	GPIOB0                             0x20000048      O        4  .data
	GPIOA0                             0x2000004c      O        4  .data
	ADC0                               0x20000050      O        4  .data
	TKEYBUF                            0x20000054      O        4  .data
	TKEY                               0x20000058      O        4  .data
	SYSCON                             0x2000005c      O        4  .data
	IFC                                0x20000060      O        4  .data
	CK801                              0x20000064      O        4  .data
	s_tkey                             0x20000068      O        4  .data
	samp_setover_f                     0x2000006c      O        1  .data
	tk_overflow_en                     0x2000006d      O        1  .data
	tk_div                             0x2000006e      O       34  .data
	neg_build_bounce                   0x20000090      O        1  .data
	pos_build_bounce                   0x20000091      O        1  .data
	tk_scan_para0                      0x20000094      O        4  .data
	scan_step_temp                     0x20000098      O        1  .data
	_end_data                          0x2000009c               0  .data
	_bss_start                         0x2000009c               0  .bss
	SysTick_100us                      0x200000a0      O        4  .bss
	SysTick_1ms                        0x200000a4      O        4  .bss
	RS485_Comming                      0x200000a8      O        4  .bss
	RS485_Comm_Flag                    0x200000ac      O        4  .bss
	RS485_Comm_Start                   0x200000b0      O        4  .bss
	RS485_Comm_End                     0x200000b4      O        4  .bss
	Press_debounce_data                0x200000bc      O        1  .bss
	TK_Lowpower_mode                   0x200000bd      O        1  .bss
	TK_Lowpower_level                  0x200000be      O        1  .bss
	TK_longpress_time                  0x200000c0      O        4  .bss
	Release_debounce_data              0x200000c4      O        1  .bss
	Key_mode                           0x200000c5      O        1  .bss
	TK_icon                            0x200000c6      O       34  .bss
	MultiTimes_Filter                  0x200000e8      O        1  .bss
	Base_Speed                         0x200000e9      O        1  .bss
	TK_IO_ENABLE                       0x200000ec      O        4  .bss
	Valid_Key_Num                      0x200000f0      O        1  .bss
	TK_senprd                          0x200000f2      O       34  .bss
	TK_Wakeup_level                    0x20000114      O        1  .bss
	TK_Triggerlevel                    0x20000116      O       34  .bss
	TK_EC_LEVEL                        0x20000138      O        2  .bss
	TK_FVR_LEVEL                       0x2000013a      O        2  .bss
	TK_BaseCnt                         0x2000013c      O        4  .bss
	TK_PSEL_MODE                       0x20000140      O        2  .bss
	R_CMPB_BUF                         0x20000144      O        4  .bss
	R_CMPA_BUF                         0x20000148      O        4  .bss
	R_SIORX_buf                        0x2000014c      O       40  .bss
	g_uart                             0x20000174      O      160  .bss
	g_uart1                            0x20000214      O      160  .bss
	m_send                             0x200002b4      O      164  .bss
	g_Dip                              0x20000358      O       16  .bss
	c_rly                              0x20000368      O       22  .bss
	baseline_data0                     0x20000380      O       34  .bss
	TK_Postive_build2                  0x200003a2      O       17  .bss
	Key_Map1                           0x200003b4      O        4  .bss
	offset_data2_abs                   0x200003b8      O       34  .bss
	scan_f                             0x200003da      O        1  .bss
	offset_data1_abs                   0x200003dc      O       34  .bss
	Release_debounce0                  0x200003fe      O       17  .bss
	Key_Map0                           0x20000410      O        4  .bss
	bsae_over_f                        0x20000414      O        1  .bss
	scan_cnt                           0x20000416      O        2  .bss
	Press_debounce0                    0x20000418      O       17  .bss
	offset_data0                       0x2000042a      O       34  .bss
	sampling_data1                     0x2000044c      O       34  .bss
	Key_Map2                           0x20000470      O        4  .bss
	Release_debounce1                  0x20000474      O       17  .bss
	tk_overflow_f                      0x20000485      O        1  .bss
	TK_Negtive_build2                  0x20000486      O       17  .bss
	base_update_f                      0x20000497      O        1  .bss
	TK_Postive_build1                  0x20000498      O       17  .bss
	time_cnt                           0x200004ac      O        4  .bss
	lpt_scan_pend_cnt                  0x200004b0      O        2  .bss
	TK_track_cnt                       0x200004b2      O        1  .bss
	Key_Map                            0x200004b4      O        4  .bss
	baseline_data1                     0x200004b8      O       34  .bss
	TK_Postive_build0                  0x200004da      O       17  .bss
	sampling_data2                     0x200004ec      O       34  .bss
	offset_data1                       0x2000050e      O       34  .bss
	TK_ovrdect_cnt                     0x20000530      O        1  .bss
	Press_debounce2                    0x20000531      O       17  .bss
	TK_Negtive_build1                  0x20000542      O       17  .bss
	tk_num                             0x20000553      O        1  .bss
	TK_Negtive_build0                  0x20000554      O       17  .bss
	Press_debounce1                    0x20000565      O       17  .bss
	Release_debounce2                  0x20000576      O       17  .bss
	r_Key_Map_Temp                     0x20000588      O        4  .bss
	tk_seque                           0x2000058c      O       17  .bss
	scan_step                          0x2000059d      O        1  .bss
	baseline_data2                     0x2000059e      O       34  .bss
	tk_sampling_max                    0x200005c0      O       34  .bss
	offset_data0_abs                   0x200005e2      O       34  .bss
	offset_data2                       0x20000604      O       34  .bss
	sampling_data0                     0x20000626      O       34  .bss
	_ebss                              0x20000648               0  .bss
	_end                               0x20000648               0  .bss
	end                                0x20000648               0  .bss
	__kernel_stack                     0x20000ff8               0  .text

	(w:Weak    d:Deubg    F:Function    f:File name    O:Zero)


======================================================================

Memory Map of the image

    Image Entry point : 0x0000010c

    Region ROM (Base: 0x00000000, Size: 0x00004560, Max: 0x00010000)

    Base Addr    Size         Type   Attr      Idx   Section Name       Object
    0x00000000   0x000001b4   Code   RO         16  .text          	Obj/arch_crt0.o
    0x000001b4   0x000009aa   Code   RO       1003  .text          	pow.o
    0x00000b5e   0x00000006   Code   RO       1011  .text          	fabs.o
    0x00000b64   0x00000020   Code   RO       1017  .text          	scalbn.o
    0x00000b84   0x00000178   Code   RO       1024  .text          	sqrt.o
    0x00000cfc   0x00000014   Code   RO       1035  .text          	_csky_case_uqi.o
    0x00000d10   0x00000038   Code   RO       1040  .text          	_fixunsdfsi.o
    0x00000d48   0x0000033a   Code   RO       1047  .text          	_addsub_df.o
    0x00001082   0x00000002   PAD
    0x00001084   0x00000234   Code   RO       1054  .text          	_mul_df.o
    0x000012b8   0x00000154   Code   RO       1061  .text          	_div_df.o
    0x0000140c   0x0000003c   Code   RO       1068  .text          	_gt_df.o
    0x00001448   0x0000003c   Code   RO       1075  .text          	_ge_df.o
    0x00001484   0x0000003a   Code   RO       1082  .text          	_le_df.o
    0x000014be   0x00000002   PAD
    0x000014c0   0x00000070   Code   RO       1089  .text          	_si_to_df.o
    0x00001530   0x00000070   Code   RO       1096  .text          	_df_to_si.o
    0x000015a0   0x00000054   Code   RO       1110  .text          	_usi_to_df.o
    0x000015f4   0x00000044   Code   RO       1117  .text          	_muldi3.o
    0x00001638   0x00000040   Code   RO       1124  .text          	_clzsi2.o
    0x00001678   0x0000019c   Code   RO       1130  .text          	_pack_df.o
    0x00001814   0x000000c4   Code   RO       1137  .text          	_unpack_df.o
    0x000018d8   0x0000008c   Code   RO       1144  .text          	_fpcmp_parts_df.o
    0x00001964   0x00000088   Code   RO       1165  .text          	memset_fast.o
    0x000019ec   0x00000064   Code   RO       1170  .text          	memcpy_fast.o
    0x00001a50   0x00000038   Code   RO         28  .text.__main   	Obj/arch_mem_init.o
    0x00001a88   0x00000074   Code   RO         61  .text.SYSCON_General_CMD.part.0	Obj/FWlib_apt32f102_syscon.o
    0x00001afc   0x0000004c   Code   RO         62  .text.SYSCON_RST_VALUE	Obj/FWlib_apt32f102_syscon.o
    0x00001b48   0x00000030   Code   RO         64  .text.SYSCON_General_CMD	Obj/FWlib_apt32f102_syscon.o
    0x00001b78   0x00000088   Code   RO         65  .text.SystemCLK_HCLKDIV_PCLKDIV_Config	Obj/FWlib_apt32f102_syscon.o
    0x00001c00   0x00000028   Code   RO         68  .text.SYSCON_HFOSC_SELECTE	Obj/FWlib_apt32f102_syscon.o
    0x00001c28   0x0000003c   Code   RO         69  .text.SYSCON_WDT_CMD	Obj/FWlib_apt32f102_syscon.o
    0x00001c64   0x00000014   Code   RO         70  .text.SYSCON_IWDCNT_Reload	Obj/FWlib_apt32f102_syscon.o
    0x00001c78   0x00000018   Code   RO         71  .text.SYSCON_IWDCNT_Config	Obj/FWlib_apt32f102_syscon.o
    0x00001c90   0x00000020   Code   RO         72  .text.SYSCON_LVD_Config	Obj/FWlib_apt32f102_syscon.o
    0x00001cb0   0x0000001c   Code   RO         73  .text.LVD_Int_Enable	Obj/FWlib_apt32f102_syscon.o
    0x00001ccc   0x0000001c   Code   RO         75  .text.IWDT_Int_Enable	Obj/FWlib_apt32f102_syscon.o
    0x00001ce8   0x00000040   Code   RO         78  .text.EXTI_trigger_CMD	Obj/FWlib_apt32f102_syscon.o
    0x00001d28   0x00000034   Code   RO         79  .text.EXTI_interrupt_CMD	Obj/FWlib_apt32f102_syscon.o
    0x00001d5c   0x00000004   Code   RO         80  .text.GPIO_EXTI_interrupt	Obj/FWlib_apt32f102_syscon.o
    0x00001d60   0x00000010   Code   RO         91  .text.EXI4_Int_Enable	Obj/FWlib_apt32f102_syscon.o
    0x00001d70   0x0000000c   Code   RO        103  .text.SYSCON_Int_Enable	Obj/FWlib_apt32f102_syscon.o
    0x00001d7c   0x0000000c   Code   RO        104  .text.SYSCON_Int_Disable	Obj/FWlib_apt32f102_syscon.o
    0x00001d88   0x00000024   Code   RO        112  .text.SYSCON_INT_Priority	Obj/FWlib_apt32f102_syscon.o
    0x00001dac   0x00000030   Code   RO        113  .text.Set_INT_Priority	Obj/FWlib_apt32f102_syscon.o
    0x00001ddc   0x000000e0   Code   RO        132  .text.GPIO_Init	Obj/FWlib_apt32f102_gpio.o
    0x00001ebc   0x00000014   Code   RO        135  .text.GPIO_PullHigh_Init	Obj/FWlib_apt32f102_gpio.o
    0x00001ed0   0x0000000e   Code   RO        141  .text.GPIO_DriveStrength_EN	Obj/FWlib_apt32f102_gpio.o
    0x00001ee0   0x0000010c   Code   RO        143  .text.GPIO_IntGroup_Set	Obj/FWlib_apt32f102_gpio.o
    0x00001fec   0x000000fc   Code   RO        144  .text.GPIOA0_EXI_Init	Obj/FWlib_apt32f102_gpio.o
    0x000020e8   0x00000008   Code   RO        147  .text.GPIO_Write_High	Obj/FWlib_apt32f102_gpio.o
    0x000020f0   0x00000008   Code   RO        148  .text.GPIO_Write_Low	Obj/FWlib_apt32f102_gpio.o
    0x000020f8   0x00000016   Code   RO        150  .text.GPIO_Reverse	Obj/FWlib_apt32f102_gpio.o
    0x0000210e   0x00000010   Code   RO        151  .text.GPIO_Read_Status	Obj/FWlib_apt32f102_gpio.o
    0x00002120   0x00000014   Code   RO        185  .text.LPT_Soft_Reset	Obj/FWlib_apt32f102_lpt.o
    0x00002134   0x00000010   Code   RO        234  .text.WWDT_CNT_Load	Obj/FWlib_apt32f102_wwdt.o
    0x00002144   0x0000001c   Code   RO        303  .text.BT_DeInit	Obj/FWlib_apt32f102_bt.o
    0x00002160   0x00000008   Code   RO        305  .text.BT_Start 	Obj/FWlib_apt32f102_bt.o
    0x00002168   0x0000000a   Code   RO        309  .text.BT_Soft_Reset	Obj/FWlib_apt32f102_bt.o
    0x00002172   0x00000018   Code   RO        310  .text.BT_Configure	Obj/FWlib_apt32f102_bt.o
    0x0000218a   0x0000002c   Code   RO        311  .text.BT_ControlSet_Configure	Obj/FWlib_apt32f102_bt.o
    0x000021b6   0x00000006   Code   RO        312  .text.BT_Period_CMP_Write	Obj/FWlib_apt32f102_bt.o
    0x000021bc   0x00000012   Code   RO        319  .text.BT_ConfigInterrupt_CMD	Obj/FWlib_apt32f102_bt.o
    0x000021d0   0x00000010   Code   RO        322  .text.BT1_INT_ENABLE	Obj/FWlib_apt32f102_bt.o
    0x000021e0   0x000000a0   Code   RO        340  .text.GPT_IO_Init	Obj/FWlib_apt32f102_gpt.o
    0x00002280   0x00000014   Code   RO        341  .text.GPT_Configure	Obj/FWlib_apt32f102_gpt.o
    0x00002294   0x00000044   Code   RO        342  .text.GPT_WaveCtrl_Configure	Obj/FWlib_apt32f102_gpt.o
    0x000022d8   0x00000014   Code   RO        343  .text.GPT_WaveLoad_Configure	Obj/FWlib_apt32f102_gpt.o
    0x000022ec   0x000000b4   Code   RO        344  .text.GPT_WaveOut_Configure	Obj/FWlib_apt32f102_gpt.o
    0x000023a0   0x00000010   Code   RO        353  .text.GPT_Start	Obj/FWlib_apt32f102_gpt.o
    0x000023b0   0x00000010   Code   RO        360  .text.GPT_Period_CMP_Write	Obj/FWlib_apt32f102_gpt.o
    0x000023c0   0x0000001c   Code   RO        365  .text.GPT_ConfigInterrupt_CMD	Obj/FWlib_apt32f102_gpt.o
    0x000023dc   0x00000018   Code   RO        435  .text.UART0_DeInit	Obj/FWlib_apt32f102_uart.o
    0x000023f4   0x00000018   Code   RO        436  .text.UART1_DeInit	Obj/FWlib_apt32f102_uart.o
    0x0000240c   0x00000018   Code   RO        437  .text.UART2_DeInit	Obj/FWlib_apt32f102_uart.o
    0x00002424   0x0000001c   Code   RO        440  .text.UART1_Int_Enable	Obj/FWlib_apt32f102_uart.o
    0x00002440   0x0000001c   Code   RO        442  .text.UART2_Int_Enable	Obj/FWlib_apt32f102_uart.o
    0x0000245c   0x000000ec   Code   RO        450  .text.UART_IO_Init	Obj/FWlib_apt32f102_uart.o
    0x00002548   0x00000010   Code   RO        452  .text.UARTInitRxTxIntEn	Obj/FWlib_apt32f102_uart.o
    0x00002558   0x0000001e   Code   RO        456  .text.UARTTransmit	Obj/FWlib_apt32f102_uart.o
    0x00002578   0x00000028   Code   RO        516  .text.EPT_Stop 	Obj/FWlib_apt32f102_ept.o
    0x000025a0   0x00000024   Code   RO        690  .text.startup.main	Obj/main.o
    0x000025c4   0x0000002c   Code   RO        707  .text.delay_nms	Obj/mcu_initial.o
    0x000025f0   0x00000022   Code   RO        708  .text.delay_nus	Obj/mcu_initial.o
    0x00002614   0x00000060   Code   RO        712  .text.BT_CONFIG	Obj/mcu_initial.o
    0x00002674   0x00000062   Code   RO        718  .text.SYSCON_CONFIG	Obj/mcu_initial.o
    0x000026d8   0x0000004c   Code   RO        719  .text.APT32F102_init	Obj/mcu_initial.o
    0x00002724   0x000000f0   Code   RO        735  .text.SYSCONIntHandler	Obj/mcu_interrupt.o
    0x00002814   0x00000068   Code   RO        736  .text.IFCIntHandler	Obj/mcu_interrupt.o
    0x0000287c   0x00000068   Code   RO        737  .text.ADCIntHandler	Obj/mcu_interrupt.o
    0x000028e4   0x000001ac   Code   RO        738  .text.EPT0IntHandler	Obj/mcu_interrupt.o
    0x00002a90   0x00000034   Code   RO        739  .text.WWDTHandler	Obj/mcu_interrupt.o
    0x00002ac4   0x00000080   Code   RO        740  .text.GPT0IntHandler	Obj/mcu_interrupt.o
    0x00002b44   0x00000070   Code   RO        741  .text.RTCIntHandler	Obj/mcu_interrupt.o
    0x00002bb4   0x0000003c   Code   RO        742  .text.UART0IntHandler	Obj/mcu_interrupt.o
    0x00002bf0   0x00000094   Code   RO        743  .text.UART1IntHandler	Obj/mcu_interrupt.o
    0x00002c84   0x0000004c   Code   RO        744  .text.UART2IntHandler	Obj/mcu_interrupt.o
    0x00002cd0   0x000000e8   Code   RO        745  .text.SPI0IntHandler	Obj/mcu_interrupt.o
    0x00002db8   0x00000054   Code   RO        746  .text.SIO0IntHandler	Obj/mcu_interrupt.o
    0x00002e0c   0x00000030   Code   RO        747  .text.EXI0IntHandler	Obj/mcu_interrupt.o
    0x00002e3c   0x00000030   Code   RO        748  .text.EXI1IntHandler	Obj/mcu_interrupt.o
    0x00002e6c   0x00000048   Code   RO        749  .text.EXI2to3IntHandler	Obj/mcu_interrupt.o
    0x00002eb4   0x00000020   Code   RO        750  .text.EXI4to9IntHandler	Obj/mcu_interrupt.o
    0x00002ed4   0x0000006c   Code   RO        751  .text.EXI10to15IntHandler	Obj/mcu_interrupt.o
    0x00002f40   0x00000034   Code   RO        752  .text.LPTIntHandler	Obj/mcu_interrupt.o
    0x00002f74   0x0000004c   Code   RO        753  .text.BT0IntHandler	Obj/mcu_interrupt.o
    0x00002fc0   0x00000070   Code   RO        754  .text.BT1IntHandler	Obj/mcu_interrupt.o
    0x00003030   0x00000002   Code   RO        755  .text.PriviledgeVioHandler	Obj/mcu_interrupt.o
    0x00003032   0x00000008   Code   RO        757  .text.PendTrapHandler	Obj/mcu_interrupt.o
    0x0000303a   0x00000008   Code   RO        758  .text.Trap3Handler	Obj/mcu_interrupt.o
    0x00003042   0x00000008   Code   RO        759  .text.Trap2Handler	Obj/mcu_interrupt.o
    0x0000304a   0x00000008   Code   RO        760  .text.Trap1Handler	Obj/mcu_interrupt.o
    0x00003052   0x00000008   Code   RO        761  .text.Trap0Handler	Obj/mcu_interrupt.o
    0x0000305a   0x00000008   Code   RO        762  .text.UnrecExecpHandler	Obj/mcu_interrupt.o
    0x00003062   0x00000008   Code   RO        763  .text.BreakPointHandler	Obj/mcu_interrupt.o
    0x0000306a   0x00000008   Code   RO        764  .text.AccessErrHandler	Obj/mcu_interrupt.o
    0x00003072   0x00000008   Code   RO        765  .text.IllegalInstrHandler	Obj/mcu_interrupt.o
    0x0000307a   0x00000008   Code   RO        766  .text.MisalignedHandler	Obj/mcu_interrupt.o
    0x00003082   0x00000008   Code   RO        767  .text.CNTAIntHandler	Obj/mcu_interrupt.o
    0x0000308a   0x00000008   Code   RO        768  .text.I2CIntHandler	Obj/mcu_interrupt.o
    0x00003094   0x00000024   Code   RO        785  .text.__divsi3 	Obj/drivers_apt32f102.o
    0x000030b8   0x00000024   Code   RO        786  .text.__udivsi3	Obj/drivers_apt32f102.o
    0x000030dc   0x00000024   Code   RO        788  .text.__umodsi3	Obj/drivers_apt32f102.o
    0x00003100   0x00000006   Code   RO        806  .text.CK_CPU_EnAllNormalIrq	Obj/drivers_apt32f102_ck801.o
    0x00003106   0x00000006   Code   RO        807  .text.CK_CPU_DisAllNormalIrq	Obj/drivers_apt32f102_ck801.o
    0x0000310c   0x00000120   Code   RO        821  .text.UARTx_Init	Obj/SYSTEM_uart.o
    0x0000322c   0x00000034   Code   RO        823  .text.UART1_RecvINT_Processing	Obj/SYSTEM_uart.o
    0x00003260   0x00000060   Code   RO        824  .text.UART1_TASK	Obj/SYSTEM_uart.o
    0x000032c0   0x000000c4   Code   RO        830  .text.BUS485_Send	Obj/SYSTEM_uart.o
    0x00003384   0x00000064   Code   RO        831  .text.MultSend_Task	Obj/SYSTEM_uart.o
    0x000033e8   0x0000005c   Code   RO        832  .text.Set_GroupSend	Obj/SYSTEM_uart.o
    0x00003444   0x0000002c   Code   RO        835  .text.BUS485Send_Task	Obj/SYSTEM_uart.o
    0x00003470   0x0000003c   Code   RO        837  .text.BusIdle_Task	Obj/SYSTEM_uart.o
    0x000034ac   0x00000054   Code   RO        838  .text.BusBusy_Task	Obj/SYSTEM_uart.o
    0x00003500   0x0000000c   Code   RO        840  .text.Dbg_Println	Obj/SYSTEM_uart.o
    0x0000350c   0x00000034   Code   RO        858  .text.DIP_GetSwitchState	Obj/SYSTEM_dip_switch.o
    0x00003540   0x0000008c   Code   RO        859  .text.DIP_Switch_Init	Obj/SYSTEM_dip_switch.o
    0x000035cc   0x0000008c   Code   RO        860  .text.DIP_ScanTask	Obj/SYSTEM_dip_switch.o
    0x00003658   0x000000cc   Code   RO        878  .text.Relay_Init	Obj/SYSTEM_control_rly.o
    0x00003724   0x00000016   Code   RO        879  .text.CheckSum 	Obj/SYSTEM_control_rly.o
    0x0000373c   0x0000001c   Code   RO        881  .text.Change_OUTV	Obj/SYSTEM_control_rly.o
    0x00003758   0x00000090   Code   RO        882  .text.BLV_VolOut_Ctrl	Obj/SYSTEM_control_rly.o
    0x000037e8   0x0000007c   Code   RO        883  .text.BLV_RLY_Ctrl_Purpose	Obj/SYSTEM_control_rly.o
    0x00003864   0x00000054   Code   RO        884  .text.BLV_RLY_Task	Obj/SYSTEM_control_rly.o
    0x000038b8   0x0000009c   Code   RO        885  .text.BLV_A9RLY_CMD_SET_Processing	Obj/SYSTEM_control_rly.o
    0x00003954   0x00000078   Code   RO        886  .text.BLV_A9RLY_CMD_READ_Processing	Obj/SYSTEM_control_rly.o
    0x000039cc   0x000000b0   Code   RO        888  .text.BLV_RLY_RS485_Pro	Obj/SYSTEM_control_rly.o
    0x00003a7c   0x00000058   Code   RO        949  .text.TK_Sampling_prog	FWlib_apt32f102_tkey_c_1_17.o
    0x00003ad4   0x00000088   Code   RO        953  .text.TKEYIntHandler	FWlib_apt32f102_tkey_c_1_17.o
    0x00003b5c   0x00000028   Code   RO        954  .text.get_key_number	FWlib_apt32f102_tkey_c_1_17.o
    0x00003b84   0x00000020   Code   RO        956  .text.TK_Scan_Start	FWlib_apt32f102_tkey_c_1_17.o
    0x00003ba4   0x00000180   Code   RO        957  .text.TK_Keymap_prog	FWlib_apt32f102_tkey_c_1_17.o
    0x00003d24   0x0000011c   Code   RO        958  .text.TK_overflow_predict	FWlib_apt32f102_tkey_c_1_17.o
    0x00003e40   0x000001d0   Code   RO        959  .text.TK_Baseline_tracking	FWlib_apt32f102_tkey_c_1_17.o
    0x00004010   0x00000054   Code   RO        960  .text.TK_result_prog	FWlib_apt32f102_tkey_c_1_17.o
    0x00004064   0x00000078   Code   RO        961  .text.CORETHandler	FWlib_apt32f102_tkey_c_1_17.o
    0x000040dc   0x00000284   Code   RO        983  .text.std_clk_calib	FWlib_apt32f102_clkcalib.o
    0x00004360   0x00000030   Data   RO       1006  .rodata        	pow.o
    0x00004390   0x00000014   Data   RO       1106  .rodata        	_thenan_df.o
    0x000043a4   0x00000100   Data   RO       1154  .rodata        	_clz.o
    0x000044a4   0x0000000b   Data   RO        691  .rodata.str1.1 	Obj/main.o
    0x000044af   0x0000000c   Data   RO        861  .rodata.str1.1 	Obj/SYSTEM_dip_switch.o
    0x000044bb   0x000000a4   Data   RO        890  .rodata.str1.1 	Obj/SYSTEM_control_rly.o
    0x0000455f   0x00000001   PAD

    Region RAM (Base: 0x20000000, Size: 0x00000648, Max: 0x00001000)

    Base Addr    Size         Type   Attr      Idx   Section Name       Object
    0x20000000   0x00000068   Data   RW        783  .data          	Obj/drivers_apt32f102.o
    0x20000068   0x00000031   Data   RW        940  .data          	FWlib_apt32f102_tkey_c_1_17.o
    0x20000099   0x00000003   PAD
    0x2000009c   0x0000000c   Zero   RW        734  .bss           	Obj/mcu_interrupt.o
    0x200000a8   0x00000010   Zero   RW        820  .bss           	Obj/SYSTEM_uart.o
    0x200000b8   0x00000004   Zero   RW        857  .bss           	Obj/SYSTEM_dip_switch.o
    0x200000bc   0x00000086   Zero   RW        703  COMMON         	Obj/main.o
    0x20000142   0x00000002   PAD
    0x20000144   0x00000030   Zero   RW        781  COMMON         	Obj/mcu_interrupt.o
    0x20000174   0x000001e4   Zero   RW        854  COMMON         	Obj/SYSTEM_uart.o
    0x20000358   0x00000010   Zero   RW        874  COMMON         	Obj/SYSTEM_dip_switch.o
    0x20000368   0x00000016   Zero   RW        903  COMMON         	Obj/SYSTEM_control_rly.o
    0x2000037e   0x00000002   PAD
    0x20000380   0x000002c8   Zero   RW        979  COMMON         	FWlib_apt32f102_tkey_c_1_17.o

    Region *default* (Base: 0x00000000, Size: 0x00000000, Max: 0xffffffff)


======================================================================

Image component sizes

       Code    RO Data    RW Data    ZI Data      Debug   Object Name

          0          0          0          0          0   linker stubs
        436          0          0          0        286   Obj/arch_crt0.o
         56          0          0          0        820   Obj/arch_mem_init.o
          0          0          0          0          0   Obj/arch_apt32f102_iostring.o
        852          0          0          0      21127   Obj/FWlib_apt32f102_syscon.o
        832          0          0          0      13094   Obj/FWlib_apt32f102_gpio.o
         20          0          0          0      13494   Obj/FWlib_apt32f102_lpt.o
          0          0          0          0          0   Obj/FWlib_apt32f102_crc.o
         16          0          0          0       8327   Obj/FWlib_apt32f102_wwdt.o
          0          0          0          0          0   Obj/FWlib_apt32f102_countera.o
          0          0          0          0          0   Obj/FWlib_apt32f102_et.o
        154          0          0          0      11840   Obj/FWlib_apt32f102_bt.o
        508          0          0          0      21406   Obj/FWlib_apt32f102_gpt.o
          0          0          0          0          0   Obj/FWlib_apt32f102_sio.o
          0          0          0          0          0   Obj/FWlib_apt32f102_spi.o
        410          0          0          0      11721   Obj/FWlib_apt32f102_uart.o
          0          0          0          0          0   Obj/FWlib_apt32f102_i2c.o
         40          0          0          0      28174   Obj/FWlib_apt32f102_ept.o
          0          0          0          0          0   Obj/FWlib_apt32f102_rtc.o
          0          0          0          0          0   Obj/FWlib_apt32f102_adc.o
          0          0          0          0          0   Obj/FWlib_apt32f102_ifc.o
          0          0          0          0          0   Obj/FWlib_apt32f102_coret.o
         36         11          0        134      11713   Obj/main.o
        348          0          0          0      15894   Obj/mcu_initial.o
       2414          0          0         60      14791   Obj/mcu_interrupt.o
        108          0        104          0       8379   Obj/drivers_apt32f102.o
         12          0          0          0       8319   Obj/drivers_apt32f102_ck801.o
       1024          0          0        500      15080   Obj/SYSTEM_uart.o
        332         12          0         20      10898   Obj/SYSTEM_dip_switch.o
       1058        164          0         22      14912   Obj/SYSTEM_control_rly.o
          0          0          0          0          0   Obj/SYSTEM_eeprom.o
          0          0          0          0          0   Obj/__rt_entry.o
	------------------------------------------------------------
       8656        187        104        736     230275   Object Totals
          4          1          3          4          0   Pad
          0          0          0          0          0   LD_GEN

	------------------------------------------------------------
    [Library Name]: .\lib_102TKey_c_1_16P0.a
	------------------------------------------------------------
       Code    RO Data    RW Data    ZI Data      Debug   Library Member Name

       1632          0         49        712      16345   FWlib_apt32f102_tkey_c_1_17.o
	------------------------------------------------------------
       1632          0         49        712      16345   Library Totals
          0          0          0          0          0   Pad
          0          0          0          0          0   LD_GEN

	------------------------------------------------------------
    [Library Name]: .\lib_102ClkCalib_1_03.a
	------------------------------------------------------------
       Code    RO Data    RW Data    ZI Data      Debug   Library Member Name

        644          0          0          0       8675   FWlib_apt32f102_clkcalib.o
	------------------------------------------------------------
        644          0          0          0       8675   Library Totals
          0          0          0          0          0   Pad
          0          0          0          0          0   LD_GEN

	------------------------------------------------------------
    [Library Name]: d:/app/cdkrepo/toolchain/ckv2elfminilib/v3.10.29/r/bin/../lib/gcc/csky-elfabiv2/6.3.0/../../../../csky-elfabiv2/lib/ck801\libm.a
	------------------------------------------------------------
       Code    RO Data    RW Data    ZI Data      Debug   Library Member Name

       2474         48          0          0          0   pow.o
          6          0          0          0          0   fabs.o
         32          0          0          0          0   scalbn.o
        376          0          0          0          0   sqrt.o
	------------------------------------------------------------
       2888         48          0          0          0   Library Totals
          0          0          0          0          0   Pad
          0          0          0          0          0   LD_GEN

	------------------------------------------------------------
    [Library Name]: d:/app/cdkrepo/toolchain/ckv2elfminilib/v3.10.29/r/bin/../lib/gcc/csky-elfabiv2/6.3.0/ck801\libgcc.a
	------------------------------------------------------------
       Code    RO Data    RW Data    ZI Data      Debug   Library Member Name

         20          0          0          0          0   _csky_case_uqi.o
         56          0          0          0          0   _fixunsdfsi.o
        826          0          0          0          0   _addsub_df.o
        564          0          0          0          0   _mul_df.o
        340          0          0          0          0   _div_df.o
         60          0          0          0          0   _gt_df.o
         60          0          0          0          0   _ge_df.o
         58          0          0          0          0   _le_df.o
        112          0          0          0          0   _si_to_df.o
        112          0          0          0          0   _df_to_si.o
          0         20          0          0          0   _thenan_df.o
         84          0          0          0          0   _usi_to_df.o
         68          0          0          0          0   _muldi3.o
         64          0          0          0          0   _clzsi2.o
        412          0          0          0          0   _pack_df.o
        196          0          0          0          0   _unpack_df.o
        140          0          0          0          0   _fpcmp_parts_df.o
          0        256          0          0          0   _clz.o
	------------------------------------------------------------
       3172        276          0          0          0   Library Totals
          0          0          0          0          0   Pad
          0          0          0          0          0   LD_GEN

	------------------------------------------------------------
    [Library Name]: d:/app/cdkrepo/toolchain/ckv2elfminilib/v3.10.29/r/bin/../lib/gcc/csky-elfabiv2/6.3.0/../../../../csky-elfabiv2/lib/ck801\libc.a
	------------------------------------------------------------
       Code    RO Data    RW Data    ZI Data      Debug   Library Member Name

        136          0          0          0          0   memset_fast.o
        100          0          0          0          0   memcpy_fast.o
          0          0          0          0          0   strncmp.o
	------------------------------------------------------------
        236          0          0          0          0   Library Totals
          0          0          0          0          0   Pad
          0          0          0          0          0   LD_GEN

	------------------------------------------------------------

======================================================================


       Code    RO Data    RW Data    ZI Data      Debug
      17232        512        156       1452     255295   Grand Totals
      17232        512        156       1452     255295   Elf Image Totals
      17232        512        156          0          0   ROM Totals

======================================================================

Total	RO	Size (Code + RO Data)				17744 (  17.33kB)
Total	RW	Size (RW Data + ZI Data)			1608 (  1.57kB)
Total	ROM	Size (Code + RO Data + RW Data)		17900 (  17.48kB)

======================================================================
